:10000000F01F0010415100003F5100003F5100001F
:100010003F5100003F5100003F5100000000000030
:100020000000000000000000000000003F51000040
:100030003F510000000000003F510000E522000099
:10004000ED200000ED200000ED200000ED2000007C
:10005000ED200000ED200000ED200000ED2000006C
:10006000ED200000ED200000ED200000ED2000005C
:10007000ED2000003D5100003D510000C100000096
:10008000AD230000C5230000D9250000F1250000A4
:100090003D510000352700003D5100003D5100005A
:1000A0003D5100003D5100003D5100003D51000018
:1000B0003D5100003D5100003D5100003D51000008
:1000C000554B10B51A6801321A60544B1A68544BDC
:1000D000D2B2302A69D01ADC182A44D012DC082A9D
:1000E00032D0102A00D094E04E4A002111604E49CF
:1000F0000A68501C08604D49895C4D4AC9B21160BC
:10010000282287E0202A63D0282A32D081E0482A9A
:100110005ED004DC382A51D0402A53D079E0502AEE
:1001200060D0582A75D13F490A68501C0860404980
:1001300008684049C0B288543F4A0221FF3111602B
:1001400080221021D20563E0374A00211160116836
:10015000481C1060354A515C354AC9B211602822EA
:100160001A6001223CE030490A68501C08602F499F
:1001700009E02D4A314910680968884207D21168A0
:10018000481C1060294A515C294AC9B240E02C4AF7
:1001900011688022D205002901D0202138E02649AB
:1001A0000220FF300860102132E08022D2051021A9
:1001B000116008221A608122520011E08221490058
:1001C0001D4A25E01E4A1168042201291AD11DE0AA
:1001D0008022D2051021116008221A600422FF3209
:1001E000154B17E00F4A1168481C1060104804684E
:1001F0001048E4B244541068114A116804220139CD
:10020000884203D28021C9050A6002E01A6000E03A
:10021000116008221A6010BD900200100400004016
:1002200018000040840200108C020010B40400107A
:1002300008000040A404001088020010C40400104C
:10024000A00400101B4B02211A6810B50A431A6063
:10025000194B20211A68041C0A431A60174B1849CD
:100260001A680A401A601868012210431860154B7A
:1002700018680140196019680A431A60124B6C2211
:100280001A60124B1249186804F0E0FF114A10601E
:10029000114A1060022C02D1104BA0221A60104BA0
:1002A000802212021A6080234022DB0501201A609E
:1002B00010BDC046048004408080044030400440AB
:1002C000F8FCFFFF34400440180000409804001080
:1002D000400D030014000040100000400C000040DE
:1002E00000E100E0034B1B689A06FBD5024B186047
:1002F0007047C0461480004000800040FFFFFFFFB1
:100300007FB5051C00200C1C01F0E0F9002801D08D
:1003100002F0E6FD00262660281C2E60211C01F05C
:1003200003FA301C01F0D2F9B04207D002F0D8FD38
:100330002660281C2E60211C01F0F6F90C4B1B785E
:10034000002B13D00B4B2A6818680B49824203D14B
:1003500020680D68A84209D01A60236801A80B60C4
:10036000064902F019FC01A802F0BEFC7FBDC046A0
:10037000880300103C01001040010010745300007D
:1003800038B5051C0C1C281C211C01F0A7FF024BD2
:100390001B68002BF7D138BD6802001008B501F0CA
:1003A000D1FF08BD08B500230B60036001F0BCF964
:1003B00008BD000010B502F05BFD0D4B0020196870
:1003C00002F080F9002002F06DF9002002F04AF9F5
:1003D000084B01241C60084B201C198802F02EF8E1
:1003E000201C02F01BF8201C01F0F8FF10BDC046D5
:1003F00094040010800200109C04001037B50C24F7
:100400000120032101F06AFF684601A9FFF778FF88
:10041000009D002D02D1013C002CF1D1FFF7CAFF55
:10042000281C3EBD08B5002002F02CF9012001F087
:10043000E5FF02F023FD08BD38B5051C0C1CFFF7D5
:10044000B9FF054B0122281C211C5A6204F07CF8DC
:10045000FFF7E8FF38BDC046700C001010B5041C53
:10046000FFF7A8FF201C03F0DFFF041CFFF7DAFFF3
:10047000201C10BD08B50020FFF7F0FF08BD0000EC
:1004800008B5021C0249034802F07AFB08BDC046C9
:100490008A5300008253000037B500F08DFF03221D
:1004A000164B1748002101F075F800F08FFFFFF799
:1004B000E1FF1448FFF7E4FF134B144A00241A60CD
:1004C0001D1C2B689C4211DA02F016FA002803D09A
:1004D00001F0E4FC00240FE00A2001F033FF68463D
:1004E00001A9FFF70DFF009B002B05D0FFF7C2FF0E
:1004F000074802F045FB37BD0134E2E7B45C000079
:1005000093530000A25300008403001070170000F2
:10051000A8530000704700001B4B73B5041C1B4917
:10052000186804F093FE1A4900901A4A1A4B201CCE
:1005300002F032FB01F0D4F9002812D001F0ECF9FE
:10054000FA218900061C04F081FE051C201C02F023
:1005500074FB124B20186B431149F3182A1C02F04C
:100560001BFB201C02F069FB0E4B20181B68002BA4
:1005700002D003DA0C4A02E00C4A00E00C4A0D49B2
:1005800002F00AFB73BDC0469804001040420F0001
:10059000B95300008A530000C653000018FCFFFF47
:1005A000CA53000050010010B6530000B3530000BE
:1005B000BD9C0000D553000070B5051C0E1C141C1A
:1005C00000F0FAFE301C291C0022064B00F0E2FF6E
:1005D000201C01210922044B00F0DCFF00F0F6FE94
:1005E00070BDC046B45C0000AC5C000000B5084BB8
:1005F00089B01A78074B68461B78074902F0CCFA95
:1006000001206946054AFFF7D7FF09B000BDC04683
:100610004401001000000010FA53000008540000CC
:10062000F0B52A4C2A4D237885B001932F78FFF737
:10063000DDFFFFF71FFF002602A803A9FFF760FEFA
:10064000029800282BD0C0B200F0BEFF40280CD08A
:1006500004D830280ED0392817D01BE0462830D0D7
:1006600049280DD0412815D126E02B783E2B11D8F2
:10067000013303E02B78002B0CD0013B2B7009E0F9
:100680002378062B06D8013303E02378002B01D012
:10069000013B237000F07CFEFFF7A8FF0026029BC1
:1006A000002B02D0C82001F04DFE042003210136AA
:1006B000FFF766FE1D2EBFDD019B2F70237000F03B
:1006C00067FEFFF7D7FE05B0F0BDC0460000001082
:1006D0004401001038B5051C0C1C00F038FE291C24
:1006E000221C0120FFF768FF034B00225A60034AD7
:1006F000943212689A6038BD700C0010D404001057
:1007000010B590B0041C6846FFF706FF201C694630
:100710006A46FFF751FF10B010BD000000B52D2252
:100720008DB0002800D02B2268460D4902F034FA23
:1007300004A802F067FC0120694604AAFFF73CFF09
:1007400003200021FFF71CFE0220FFF787FE002890
:10075000EED00A200021FFF713FE0DB000BDC04609
:100760003B540000F8B5041C161C0D1C002702F0B9
:1007700049FC211C1431E774681C02F067FA00F090
:100780001BFE201C04213A1C0A4B00F003FF0A4CFC
:10079000281C04210922231C00F0FCFEBE4205D0C7
:1007A000064878210922231C00F0F4FE00F00EFE1A
:1007B000F8BDC046B45C0000AC5C00009D5D00006C
:1007C00010B58CB0FFF756FE124902A802F03EFAAF
:1007D00004A802A90022FFF7C5FF2E24FF3400223F
:1007E00004A802A9FFF7BEFF0020032101F076FD57
:1007F0000023684601A901930093FFF781FD009B48
:10080000002B02D1013C002CE9D1FFF733FE0CB0E4
:1008100010BDC046BE9C0000F0B5002493B0059406
:10082000FFF728FE0222962301940392271C5B0007
:10083000029300F0C1FD019B9A4E002B6DD10AADD1
:10084000281C02F0DFFB019AEA742A746A73AA7208
:10085000EA712A71002C01D1012F05D1281C042135
:100860000022331C00F096FE8F4D331C281C1E21E5
:10087000002200F08FFE8B4E012C01D1012F06D1FA
:1008800068462D3025210022331C00F083FE281CF1
:1008900033210022331C00F07DFE824D022C09D151
:1008A000012F07D0684633304D2100222B1C00F069
:1008B00071FE09E00CA83A2100222B1C00F06AFE10
:1008C000032CEFD1012FEDD0784E2B1C301C592179
:1008D000002200F05FFE734D042C01D1012F06D1E0
:1008E000684636305F2100222B1C00F053FE301C7E
:1008F0006C2100222B1C00F04DFE052C01D1012F94
:1009000006D16846393072210022664B00F042FE63
:100910000FA804210922664B03E066480421002247
:10092000331C00F037FE00F051FD059B002B0AD070
:10093000143B012B05D8052C03D0962001F002FDB5
:1009400001E0FFF797FD0320011CFFF719FD0020D0
:1009500000F0BCFE0023051C06A905A8069305931C
:10096000FFF7CEFC059B002B74D007AD08AE281C0A
:10097000311C09AA02F07AFB0190002871D1281CD1
:1009800002F05EFC071C05981238052868D804F0B0
:10099000FBFB0567240C6703601C00E0601D06215B
:1009A00004F0AAFC00270C1C5BE0601E042804D89D
:1009B00004F0EAFB060B0D103A002B88013316E019
:1009C000A8780C2104F038FC19E001375FE030789A
:1009D00001301BE07078013020E0601E042804D84C
:1009E00004F0D2FB0810121A22002B88013B2B8046
:1009F000002445E0A8780C210A3004F07DFC013188
:100A0000A9703DE0013F42E030781730182104F032
:100A100073FC0422317040E070783B303C2104F0DC
:100A20006BFC0323717030E00023B370381C072186
:100A300004F062FC281C0A1C0991311C052C02D10F
:100A400002F06FFB02E0039B02F02AFB01279623D2
:100A5000BB4008E0002D07D101235F401F4003E0A9
:100A6000012796235B000293059B842B17D0182B3C
:100A700015D0029B029A013B002A00D0D8E60EE076
:100A8000281C02F0DDFB0523071C0393CEE7381C6E
:100A9000291C02F005FC022405220392C6E713B0CC
:100AA000F0BDC046B45C000044540000395400005E
:100AB000AC5C000046540000F7B502F039FA18208B
:100AC0000021FFF7B9FC0024694EFFF7ABFC694D2C
:100AD00000236B62201C02F04CFA002C02D0002094
:100AE000012101E00620032101F0F8FB201C02F0A7
:100AF0003BFA01A9071C6846002F03D0FFF752FC00
:100B0000012725E0FFF74EFC009A002A20D1002C97
:100B1000E0D1594B1B68002BDCD1584B98331B6834
:100B2000002B07D1564BF618D4D500F0F9FB022460
:100B30004F4ECFE7534B00941A6811321A60009A57
:100B4000102AEFDC03F020FC009B01330093F6E752
:100B5000002C0CD0009B182B01D0002FB5D000F03A
:100B60003DFC4948FFF78CFC444B0122DA6600F05B
:100B7000E5FE02F047F9009A182A62D1019F00248D
:100B8000F8B200F021FD012601946E62172846D0CC
:100B90000CD813282BD002D8112819D04EE01528D4
:100BA0002DD016284AD1FFF73BFD4AE026282ED04B
:100BB00004D819281ED0212811D03FE0442836D06F
:100BC00045283BD1E120000102F0C4FA301C32E09C
:100BD0002E4B1B68002B34D0FFF7F2FD05E02B4BAA
:100BE0001B68002B2DD0FFF717FE009429E0FFF7BC
:100BF00053FC26E0264B1868301A00F0C5FF012090
:100C0000FFF77EFDFFF736FCFFF7F8FB19E0214BFD
:100C100005221C70204B1A7000F0BAFB11E01F4B2C
:100C20001A6801321A60052A0BD11C6009E01C48C1
:100C300002F090FA201CFFF771FD02E000230197FB
:100C40006B62FFF7B7FB0098019903F07DFC6B6ABC
:100C5000002B01D0FFF70EFC084B94331B68002BD0
:100C600003D100F05DFB01242EE704F007FA2AE728
:100C700020BF0200700C001068020010D4040010A5
:100C80000CFEFFFF940200105454000050010010AD
:100C900008000010440100100000001014010010B2
:100CA000F0F1FFFF73B502F00FF83A4C00F0D0FC02
:100CB0003948002101F08AF90021384801F086F90D
:100CC00000F09EFD00F03EFF23680726B34323603B
:100CD000236801252B4300202360021C0B2101F017
:100CE000FFF8201C2E4C102101F070F9236800221F
:100CF000B34323602368281C2360042101F0F0F82B
:100D0000201C002101F062F901F0D4F896200002C5
:100D100001F04EFD234D01235B4200202B60FFF7C5
:100D2000EFFC00232B6050240120FFF78BFA00F02A
:100D300009FF02F0C7F82B68002B05D16420043CA2
:100D400001F000FB142CEFD10020FFF7D9FC16486E
:100D500001F016FF192001F0F5FA01F0CDFD002891
:100D600002D0FFF799FB02E0013C002CF2DC02F01C
:100D700005FB03F0CFF91E2300930F2301930B48CB
:100D80000B490C4A0C4B03F0D7F90C4803F006FA58
:100D9000FFF792FE74400440984004409C40044099
:100DA00094400440500100105E540000F9500000CF
:100DB00001030000D506000094020010800200101C
:100DC000F7B500283BD00378303B5A425341C01856
:100DD0000378782B03D101301026012501E00A2683
:100DE00000250378002201922D2B02D1012301302E
:100DF000019300230278002A1BD0171C303FFCB25D
:100E0000092C02D87343DB1911E020273A43002D47
:100E100008D0171C613FFFB2052F03D81B01573ABA
:100E2000134304E0064801F0ABFE002007E0013068
:100E3000E0E7019A002A00D05B420B600120FEBD72
:100E4000685400000378202B01D10130FAE7704785
:100E5000031C303BDAB2092A01D8181C0AE020230F
:100E60001843031C613BDBB2052B01D8573801E066
:100E700001204042704770B50E1CFFF7E3FF0025CC
:100E8000041C2078002807D0FFF7E2FF002803DBCE
:100E90002D0105430134F4E73560201C70BD0000CE
:100EA00008B500F039FD011C014801F069FE08BDDC
:100EB0007654000000B589B0684602F0A3F8694690
:100EC000024801F05DFE09B000BDC046B25400000A
:100ED000F7B50F1C01A9161CFFF772FF002814D0EC
:100EE000019C0B49201C04F007FA0D1C081C64210E
:100EF00004F002FA281C3970642104F0A7F90449AF
:100F00003070201C04F0A2F901E001204042FEBD37
:100F10001027000037B50D1C48686A46694607313E
:100F20000632FFF7D5FF01AC69466A4620800132E0
:100F3000A8680231FFF7CCFF6B4618702288044B7B
:100F40009A4203D9201C694602F0EBF837BDC0462F
:100F50006B07000007B5486801A9FFF731FF019B47
:100F60003C20584302F0F6F807BD00000723584321
:100F7000054A10189C30013B04D3C25C002AFAD009
:100F8000002000E001207047D404001030B519485B
:100F900085B001F0F5FD0024651CA30719D1201CC4
:100FA000FFF7E4FF002810D0281CFFF7DFFF002820
:100FB0000BD0A01CFFF7DAFF002806D0E01CFFF7DB
:100FC000D5FF002801D004340EE00B48211C01F0AD
:100FD000D7FD211C684602F0E5F9684601F08EFE57
:100FE000064801F0CDFD2C1CFF2CD5DD01F094FE50
:100FF00005B030BD8A53000082540000BD9C000043
:1010000070B50E1CFFF71EFF0D25041C0134631E76
:101010001878FFF71DFF002806DB7055013DF5D25B
:10102000201CFFF70FFF00E0002070BD70B5444C9E
:1010300086B023680868251C002B06D1414801F0C2
:101040009FFD03F067F8012309E0012B0DD13E4914
:10105000082201F004FE002803D123680133236035
:101060006BE03A4801F08CFD5FE00378412B17D12B
:10107000374C0230211CFFF7C3FF002855D00378FE
:10108000422B52D1211C02300E31FFF7B9FF00284C
:101090004BD00378432B48D1211C02301C3103E094
:1010A000532B06D12B490230FFF7AAFF002844D169
:1010B0003BE04D2B1FD1284C0230211CFFF7A0FF35
:1010C000002832D003784E2B2FD1211C02300E3154
:1010D000FFF796FF002828D00378472B25D1023050
:1010E00001A9FFF7C8FE019B002B1EDB184A1B4815
:1010F00053651B491DE001A9FFF7BDFE04782023BD
:10110000061C9C4311D1301C02A9FFF779FF019BFB
:10111000061CE118FF2902DC02A802F059F9002E92
:1011200003D00134042CEED107E002F0F3FF0B48AA
:101130000C4901F025FD00232B6006B070BDC046B0
:10114000540200108B5400008A530000A154000088
:10115000D40400101A050010FE040010AD54000065
:10116000E2530000B754000037B54C682378002BD9
:1011700025D0201CFFF766FE01A9FFF77CFE019B2E
:10118000041C002B1BD0D8B2FF2B09DD00F038FA6D
:10119000019B051C1812C0B200F032FA019003E066
:1011A00000F02EFA002501900198002802D0291C99
:1011B000FFF742F923785A1E9341E418D6E737BD6A
:1011C000064A08B5137801214B40137001D0044939
:1011D00000E00449044801F0D3FC08BD8903001075
:1011E0005B540000BE540000C2540000064A08B51B
:1011F000137801214B40137001D0044900E00449E9
:10120000044801F0BDFC08BD880300105B540000D9
:10121000BE540000D154000007B5486801A9FFF78B
:10122000CFFD019B002B01DC01230193019B1E2BB1
:1012300001DD1E2301930199034A044B4A430448EC
:101240001A6001F09DFC07BD7017000084030010B8
:10125000E154000038B5051C002D09D0642402209B
:101260000021013C00F062FE002CF8D1013DF3E7C3
:1012700038BD70B5061C01200821021C00F080FE5C
:10128000072401200821002200F07AFE321C0125EB
:1012900022412A400020022100F072FE281C082171
:1012A0002A1C00F06DFE013CEBD270BD10B5002190
:1012B000041C0A1C022000F063FE201CFFF7D9FF6B
:1012C00010BDF0B5012385B002930023061C0393E3
:1012D00072B6002402AB1B59502040421843C0B2E2
:1012E000FFF7E4FF0020FFF7E1FF1020FFF7DEFF2C
:1012F000E020FFF7DBFF212767430025F7190220D5
:101300000021012200F03CFE785D0135FFF7B1FFBE
:10131000842DF4D10434082CDCD162B605B0F0BDC4
:1013200008B5AC20FFF7C2FFAE20FFF7BFFFA52036
:10133000FFF7BCFF08BD38B50122051C0C1C00F0EE
:10134000CFFD281C211C012200F01AFE38BD08B573
:10135000AF20FFF7ABFFA420FFF7A8FF08BD08B53B
:10136000AE20FFF7A3FF08BD10B5041CF820FFF75F
:101370009DFF201CFFF79AFF10BD10B5041C8120B3
:10138000FFF794FF3F202040FFF790FF10BD0000C3
:1013900008B5074B20201B781843FFF787FF0A206A
:1013A000FFF758FF034B1878FFF7E7FF08BDC0466B
:1013B000000000104401001008B5842202480021FA
:1013C000520001F017FC08BD8A03001008B502485E
:1013D000FFF777FF08BDC0468A03001008B501205B
:1013E0000821FFF7A8FF00200221FFF7A4FF022039
:1013F0000021FFF7A0FF02200621FFF79CFF03203A
:10140000011CFFF798FF0320011C002200F0B8FD2B
:1014100002200621002200F0B3FD06210122022055
:1014200000F0AEFDFFF7C8FFFFF7D0FFA220FFF7E7
:101430003DFFA020FFF73AFFC020FFF737FF002055
:10144000FFF792FF0A20FFF705FF4020FFF72EFF6E
:101450002C20FFF72BFF3220FFF7FCFE2E20FFF79A
:1014600025FF3220FFF7F6FE2F20FFF71FFF0A208F
:10147000FFF7F0FEFFF78CFFFFF769FF08BD0000E4
:1014800083280ED80F290CD8CB0884225343072277
:10149000C0181140034B80220A41111C1A5C1143F1
:1014A000195470478A030010F7B55B18DBB201933B
:1014B000019B994215D28425CC086C4307270F4025
:1014C000802504193D41EFB2A618B44206DA054D55
:1014D00065192B7801343B432B70F6E70131C9B213
:1014E000E6E7F7BD8A030010F0B51E1C87B0059231
:1014F000F27804915B68824201D2307845E0244A58
:10150000B478934205D10322041B54430192E4189A
:101510000CE0001B0022824204DA19780132023109
:101520005B18F8E71A789C1C5B780193A2180025D9
:1015300003922F1C019B9F4226DA0822002302926D
:1015400000937378009A9A421CDA029A082A06D10C
:10155000039B9C4218D00022257802920134EB07AD
:1015600008D5049A009BB818059AC0B29918C9B258
:10157000FFF786FF009B029A013301326D10009342
:101580000292DEE70137D5E7019807B0F0BDC0460B
:1015900005550000F7B5041C0D1C161C1F1C01F09E
:1015A0004CFB20180190019B9C420BD0832D09D845
:1015B0002078291C321C3B1CFFF796FF01302D18A8
:1015C0000134F0E7F7BD000010B50021012204232B
:1015D0000A4C0C5D844203D118010243D0B20BE0E7
:1015E000013B002B04D10132092A00DD1A1C04231F
:1015F00001312829ECD1002010BDC046CC5C000090
:101600000F23020918408000031F00D52833511E04
:101610000020032906D8242B04DC04218A1A02495D
:10162000CB18985C7047C046CC5C000038B5051CF0
:101630000024054B291CE05C044B0134C01800F069
:10164000C5FC0A2CF5D138BD085D000000400440FF
:10165000F8B50D4F3C68002C15D11020FFF7E6FFC0
:101660000A4B0022E65C1B195D78301C291C00F037
:1016700037FC0234301C291C012200F081FC142CA0
:10168000EED101233B60F8BD48010010F45C00007E
:1016900070B500240B4B0122E65C1B195D78301CF1
:1016A000291C00F01DFC0234301C291C002200F013
:1016B00067FC142CEED10020FFF7B8FF024B00228C
:1016C0001A6070BDF45C00004801001038B5051CBC
:1016D000FFF7BEFF002D09D007210122022000F0F4
:1016E000FFFB104B80211A688A431A6000200B21EF
:1016F00000F01CFC0124002805D000200B2100F084
:1017000015FC44424441002D09D00721002202204B
:1017100000F0E6FB034B80211A680A431A60201C84
:1017200038BDC046FC3F0250F0B587B0002602909D
:101730000120039104960596FFF7C8FFB04202D03E
:101740001823049301260021284C00912078617809
:10175000012200F0C5FB20786178002200F010FC27
:10176000234B9D1D012E24DC6A782F78111C381C18
:10177000019200F0DBFB002808D100991D4AB3005C
:101780008A5C103369465A5001360BE02878697834
:1017900000F0CCFB0028F0D0381C019900F0C6FB0B
:1017A0000028EAD0009A144B0132023D00929D427B
:1017B000D8D127786578381C291C002200F090FBCE
:1017C000291C381C012200F0DBFB0C4902348C423E
:1017D000BCD10020864206D0049A029B05991A606B
:1017E000039A0120116007B0F0BDC046F45C000010
:1017F000C45C0000CC5C0000C25C0000085D00001E
:1018000008B50120021C0B2100F06AFB01200B210E
:10181000002200F0B5FB03200221012200F060FB52
:1018200003200221002200F0ABFB08BD234B37B59B
:101830001A6810218A431A60214B8022196892018C
:101840000A431A60051C0B210120002200F048FB0E
:1018500001200B21002200F093FB1A4B9F211A68F4
:10186000194C8A431A601A6818491A60184B18688C
:1018700003F0ECFC8023000218432A1C20600221A4
:10188000032000F07DFB142000F05CFD2368FF22A4
:101890009343236023680F4A134323600E4B1B6856
:1018A0000193019B002BF9DA22680C4B1340236053
:1018B000FFF7A6FF01980004800D3EBD388204406A
:1018C000808004409840044000C0014000093D0071
:1018D00098040010800000012CC00140FFFFFFF8B9
:1018E00010B50C4C2068002813DA00202060FFF7A8
:1018F0009DFF0A280ADC0120FFF798FF0138C0236A
:10190000FF385B00984201D801232360FFF778FF7E
:10191000206810BD0400001008B5FFF7E1FF0028A3
:1019200001D1002007E00120FFF780FF011EF8D061
:10193000014803F08BFC08BD50BB120008B5FFF74F
:10194000CFFF00280AD0FFF7E7FFFA22031C00218F
:10195000C00FD2009A424841014B186008BDC046F2
:101960004C01001008B5074B02221A60064BA22258
:101970001960064B1A70A32258709A7000F0F2FD9D
:1019800008BDC046C4040010A0040010B404001038
:1019900008B5064B02311960054B00221A60054B51
:1019A000A2221A70587000F0DDFD08BDC4040010BA
:1019B000A0040010B404001070B5051C0E1C032414
:1019C000281C311CFFF7CEFF0223FF33984202D0C0
:1019D000013C002CF4D170BD70B5051C0E1C032415
:1019E000281C311CFFF7D4FF0223FF33984202D09A
:1019F000013C002CF4D170BD0B4B10B51C680023CA
:101A00009C420ED0094CA31CA270140A5C70140CEA
:101A1000120EDA709C70FFF7DFFF831EFF3B5A4205
:101A20005341181C10BDC04650010010B4040010F2
:101A300070B50E4C25680024A54215D00C4C160A32
:101A4000A270E670160C120E6271A371A21D2671AF
:101A50001C0A54701C0C1B0E9470D370FFF7BCFF53
:101A6000841EFF3C63425C41201C70BD500100108D
:101A7000B404001008B5064B1A6800239A4205D03A
:101A8000FFF79AFF831EFF3B5A425341181C08BDC3
:101A90005001001008B5074B00201B68834207D097
:101AA00002200721FFF788FF0238FF3843425841E0
:101AB00008BDC0465001001038B50F4B051C1B680F
:101AC0000020834217D00924641B631E062B10D804
:101AD000072C05D00948A91E0918221C01F068F836
:101AE000E8B2211CFFF778FF0238FF384342584123
:101AF00001E00120404238BD50010010B604001042
:101B0000012010B5011CFFF757FF0223FF33984255
:101B10000ED1094B01211960084B1C78230709D00D
:101B2000074B032222409A70081CFFF755FF01E083
:101B300001246442201C10BD50010010A4040010B8
:101B4000B404001008B5FFF7DBFF02200121FFF706
:101B500033FF0223FF3398420FD1084B1B787F2BB2
:101B600006D98422022007215204054BFFF760FFAB
:101B700009200421034AFFF73FFF08BDA404001019
:101B8000020114008080808010B500280CD0254B05
:101B900080211A688A431A60234B1B68D907FBD53A
:101BA000224B03221A6001E0204B1860204B0122D7
:101BB00000211A6019601A60196801221142FBD0D5
:101BC0001C4B80211A601C4A490214682143116091
:101BD0001A1C002804D1134B802419682143196072
:101BE000164B196888421CD01860002801D0144890
:101BF00000E01448116803F0DBFA134BFA21186077
:101C00008900041C03F022FB1E2358430F4BC821FC
:101C100018604901201C03F019FB0D4B186001F0FE
:101C20003DF810BD388204400C80044070800440B0
:101C300074800440788004408080044008000010D4
:101C4000006CDC02001BB700980400109404001024
:101C50009C04001008B500F035F9134B00211A68F8
:101C6000120B12031A60114B1A68120B12031A603E
:101C70000F4B1A68120B12031A600E4B1A68120BE4
:101C800012031A600C4B012219600C4B1A60196088
:101C90001A601A6801200242FBD0094B23221A6005
:101CA000FFF772FF08BDC046008000500080015061
:101CB0000080025000800350408004404480044073
:101CC0000880044038B50F490F4800F059FF0F4D08
:101CD0000024281C00F054FF0D4A0E48A158121988
:101CE000D2682B1C143400F04BFFDC2CF4D10A48D2
:101CF00000F046FF00F046FB011C084800F040FFE2
:101D000038BDC0468A530000125D0000625D0000CD
:101D10007C5E0000245D00002F5D0000515D00002E
:101D2000F0B53B4B8BB01E68041C002E01D1351C56
:101D300008E0384B02901B6801209B6854E0336830
:101D40001E79019D2378002B31D0082D33D02378C4
:101D5000202B01D10134FAE7002B28D06A1CAD00FA
:101D600008356B460192EC50FF2E4CD02278002AA9
:101D700007D0631C202A01D01C1CF7E70022227028
:101D80001C1C019A012ADCD1224E234B0C25336006
:101D9000371C013D002D2ED03B680298196800F0D9
:101DA0006FFF0028CBD03B6814333B60F1E7002D78
:101DB0001CD0022D02D0B54206D911E00398174974
:101DC00000F05EFF0028F6D1124C15482368D96850
:101DD00000F0D6FE23681348196900F0D1FE05E033
:101DE0000C4BE8B21B689B6802A99847084A136825
:101DF000002B0BD103E0281C291CFFF763FF0A48C6
:101E000000F0BEFE02E0019D0026D2E70BB0F0BD5F
:101E1000540200105C0200107C5E0000B75300000A
:101E20005E5D0000B2540000655D000038B5041C22
:101E3000164D0A2808D002D8082811D01CE00D2819
:101E400002D07F280CD017E02A68002313701048B6
:101E500000F096FE0F4C201CFFF762FF2C6013E091
:101E60000C4B2A689A420FD90B48211C00F088FEBF
:101E70002B68013B2B6007E00748211C00F080FE27
:101E80002B685A1C2A601C7038BDC04658020010CE
:101E9000625D000054010010715D000008B500F0A3
:101EA0002BFD002804D000F0FDFCFFF7BFFFF6E794
:101EB00008BD0000014A024B1A607047540100102F
:101EC00058020010044B40211A680A431A60034B61
:101ED00001221A707047C0468080044060020010E2
:101EE0000F4B70B51B78061C0C1C151C002B01D168
:101EF000FFF7E8FF701E022803D80A4B8000C35882
:101F000000E0094B1A68012D04D1A5402C1C144394
:101F10001C6003E00121A1408A431A6070BDC046E5
:101F200060020010585F00000080005038B50F4B71
:101F3000051C1B780C1C002B01D1FFF7C3FF0020F0
:101F4000032D12D8281C012203F01EF902040608F2
:101F5000074B04E0074B02E0074B00E0074B1B6810
:101F6000A2401340181C421E904138BD6002001070
:101F7000FC3F0050FC3F0150FC3F0250FC3F03502F
:101F80000F4B70B51B78061C0C1C151C002B01D1C7
:101F9000FFF798FF701E022803D80A4B8000C35831
:101FA00000E0094B1A68012D04D1A5402C1C1443F4
:101FB0001C6003E00121A1408A431A6070BDC04645
:101FC00060020010645F0000FC3F005038B5084B11
:101FD000041C1B780D1C002B01D1FFF773FF236835
:101FE00018229343236023681D43256038BDC046F3
:101FF00060020010054B3F221A60054B01221A6057
:10200000044B40211A688A431A60704724800440B8
:10201000D88004403882044008B5044B40211A6837
:102020008A431A60FFF7E6FF08BDC04638820440C5
:1020300008B500F05DFAFFF72BFB0A480021FFF717
:10204000C5FF09480021FFF7C1FF08480021FFF73D
:10205000BDFF07480021FFF7B9FF06480021FFF741
:10206000B5FF08BD0840044000400440AC400440B7
:10207000144004401C40044008B50120FEF7E2F87B
:1020800008BD000008B5124B8022DA675200DA67FB
:102090008022D200DA6780225201DA6780221201A0
:1020A000DA6780229200DA670A4A0023136001216E
:1020B000094A49421160094A1360094A1360094AF2
:1020C00001231360084A1360FFF7D6FF08BDC0461E
:1020D00004E100E0048204400882044004C000409F
:1020E0003CC0004000C000400040014008B5064B25
:1020F0001A6801321A60054B1868FFF745FDFFF7B3
:10210000C1FFC046C04608BD6402001008000010B0
:10211000F7B5071C0C1C72B6FFF78AFF524B1A6802
:10212000524B1A60002F01D0514B00E0514B524AE4
:1021300004211360514B524D1A680A431A60002360
:102140002B60A1071ED04F4B4F4A19680A401A60F6
:1021500029684E4BA2070ED5EC2252010A432A6091
:1021600080221A6052001A608022D2001A608022F7
:1021700052011A6003E0802212010A432A60802281
:1021800012011A60002F53D0414B00241C60414BB8
:10219000414E1C60414B301C1C60414B211C1C609B
:1021A000FFF714FF201C0921221CFFF799FE201CB9
:1021B0000921221CFFF7E4FE3A4B80211A683A48B5
:1021C0000A431A603368072293433360336802225C
:1021D000134333600A21784302F0EAFF334B0322B2
:1021E0001860334B1C60334B1A60334B334A196809
:1021F0000A401A601A6880210A431A60234A8B0039
:102200001360204A1168194311602A6802211343A0
:102210002B602B4B01221A602A4B19602A4B1C4958
:102220001A601C601A60186801221042FBD00A6014
:10223000264B012252421A60254B00221B68019353
:10224000244B1A6062B630BFC046214B019A1B680E
:102250009A4208D11F4B01221A601F4B1868FFF7E2
:1022600093FCFFF70FFFF7BD38820440348204402F
:10227000BF180000FF1800003082044010ED00E09D
:1022800004820440008204407FE2FFFF00E100E09E
:1022900004C0004004000140644004400440014088
:1022A0000480014080800440841E000018C000406B
:1022B00008C0004014C000403CC000400FF0FFFFC9
:1022C0007880044070800440748004400882044098
:1022D00064020010680200100800001008B5FFF743
:1022E00017FF08BD074B1A68013203D1064A11686F
:1022F000013111601A6801321A60044B1A68013208
:102300001A60704778020010740200106C0200100E
:10231000074B98420AD8074A00231360064A01383F
:102320001060064A1360064B07221A607047C046C9
:10233000FFFFFF007802001014E000E018E000E06A
:1023400010E000E00B4A10B51368002800D101200E
:10235000C1438B4208D91168994209D3591C1468AA
:1023600009188C42FAD3F6E71168C91A8142FBD3E7
:1023700010BDC04678020010014B18687047C04677
:1023800078020010064BFA211868064B10B5890038
:102390001C6802F00DFF044B5C43201810BDC046C2
:1023A000780200107402001037894100034B0122AB
:1023B0001A60034B1A6801321A60704700C000406F
:1023C0007C020010034B01221A60034B1A68013291
:1023D0001A6070470000014080020010002803D1FD
:1023E000044B01221A6003E0012801D1024B18605E
:1023F0007047C04604C0004004000140002802D1DC
:10240000044B186004E0012802D1034B00221A603B
:102410007047C04604C0004004000140002801D1BC
:10242000044B02E0012804D1034B1A6802210A433D
:102430001A60704704C000400400014010B5002934
:1024400000D1134900280DD1124B80241A68224371
:102450001A60114B03221860104B1960104B1A6060
:10246000620211E0012811D10A4B80221868520043
:1024700002431A600B4B00221A600B4B03221960B7
:102480000A4B1A6080229202094B1A6010BDC046A6
:10249000FFFF0000808004407C02001018C0004054
:1024A00014C00040800200101800014014000140D8
:1024B00000E100E080231022DB051A60094B0822AE
:1024C0001A6000238022D2051268D10604D5064A7C
:1024D000934201D00133F5E7044898429B415842AA
:1024E0007047C04618000040FF0F0000FE0F0000BC
:1024F00008B58022154B1202DA67154B6C221A6060
:10250000144B154A196800201140196019681960A8
:10251000124B19680A401A601A6804211A600122D5
:10252000FFF7DEFC002004210122FFF729FD002037
:1025300005210122FFF7D4FC012200200521FFF72D
:102540001FFD074B00221A6008BDC04604E100E0F1
:102550001800004030400440F8FCFFFF34400440C5
:1025600004800440F8B5174A174C00232360136019
:10257000164A202113608022D20511602168144A76
:10258000012903D0934203D00133F7E7934203D1EB
:10259000FFF790FF002014E00E4F00253E68013E3B
:1025A0002368FF2B0CD83B689E4204D03E68FFF79F
:1025B000E3FE051C0A35FFF7DFFE8542F0D1E7E7B1
:1025C0002068F8BD84020010880200108C02001000
:1025D000FF0F000090020010034B01221A60034B12
:1025E0001A6801321A6070470040014094020010DE
:1025F000174B70B501241C60164B1A6812191A602B
:10260000154B1A68002A22D01A68144D013A1A6034
:102610001E68002E0DD02A68201C211CFFF7B0FC7C
:102620002B68201CE31A2B602A680221FFF7A8FC04
:102630000DE01B68201C2B602A68211CFFF7A0FC02
:102640002A68201C0221FFF79BFC054B1E6070BD11
:10265000008001409C02001098020010A0020010AF
:1026600004800140002803D1044B01221A6003E0DA
:10267000012801D1024B18607047C0460440014058
:1026800004800140002802D1044B186004E00128B6
:1026900002D1034B00221A607047C046044001403B
:1026A00004800140002801D1044B02E0012804D13C
:1026B000034B1A6802210A431A6070470440014024
:1026C0000480014010B500280FD1124B80221C68F5
:1026D000920022431A60104B032218600F4B1960BE
:1026E0000F4B1A608022D20211E0012811D1094B50
:1026F00080221868D20002431A600A4B00221A6036
:10270000094B03221960094B1A6080221203084BFF
:102710001A6010BD808004409402001018400140EF
:10272000144001409C0200101880014014800140B8
:1027300000E100E008B5184B1A680E231340062B81
:102740000DD1164B9E221B68134205D0144ADBB2F2
:102750005360144B1B681EE0D9071CD501E0042B05
:1027600005D1104B1868C0B200F0B1F813E00C2B83
:1027700006D10B4B8022596852000A435A600AE086
:10278000022B08D1054B1A68054B910601D5002292
:1027900000E001229A6008BD0880004014800040DB
:1027A000A40200100080004000487047A4020010FE
:1027B000F7B52D4B2D4C8022002192030191061C70
:1027C000DA67201C902200F015FA019B0725A36010
:1027D000274B284F1A68AA431A601968012211432F
:1027E0001960254B1968A9431960196811431960CC
:1027F000224B80211868490101431960204B1A605F
:1028000083223A601F4A126819681F4B18685043A8
:1028100002F0CEFC311C000902F0CAFC1B4B102256
:102820001B491A60030A0B601A4BC0B203221860DE
:102830003A60194A1560194A1D1C10680190106809
:1028400060230340602BFAD110680123184202D0A4
:102850002B680193F8E723708022114B92031A60D2
:1028600005230B60F7BDC04604E100E0A4020010A0
:10287000A44004400C800040A840044080800440F4
:10288000988004407880044098040010288000401C
:102890000480004000800040088000401480004018
:1028A00000E100E008B5FFF77FFFC268031C1202D9
:1028B000120E8218D07BDA681202120E0132D2B2E6
:1028C0009A7352B2002A01DA00229A7308BD10B539
:1028D000041CFFF769FFC2681204120E8218D47339
:1028E000C2681204120E0132D2B2427352B2002AEE
:1028F00001DA0022427310BD08B5FFF755FFC26828
:10290000C36812021B041B0E120ED01A431E9841FC
:10291000C0B208BD70B500241D5D0619002D02D09F
:1029200005550134F8E7121B301C131C002B03DD86
:102930000170013B0130F9E7D043C0170240A018F5
:1029400070BDF7B5051C01910093561E092B01D8E7
:10295000041C0CE000980A2102F02AFC0199031CD7
:10296000321C281CFFF7EDFF071C2C1807E0671B23
:10297000002E04DD019B013E23700134F7E700982F
:102980000A2102F059FC3031781C2170FEBDF8B5E7
:102990000C1CD9175F18051C4F40561E092F12D961
:1029A000381C0A21002B03DA02F002FC434202E049
:1029B00002F0FEFB031C281C211C321CFFF7E7FF62
:1029C000041C2D1814E0002B00DA961E2A1CA919ED
:1029D000891A002902DD14700132F8E7F443E41784
:1029E00034402D19002B03DA2D232B7001340135CF
:1029F000381C0A2102F020FC30312970601CF8BD1F
:102A0000F7B5089F1E1C051C013A3B0901D1041CA7
:102A100005E00093331CFFF7F3FF2C1806E0601B62
:102A2000002A03DD2170013A0134F8E70F231F402B
:102A3000092F01D8303704E0002E01D0373700E0ED
:102A4000573727700130FEBDF0B585B0041C0291E8
:102A500001D00021017000251178002906D1029FC4
:102A60000023BD426CD22370281C6FE0029FBD4240
:102A7000F5D2252902D00132217004E051782529B0
:102A800004D12170023201350134E5E7302902D04A
:102A9000561C202100E0961C32782D3A50424241CB
:102AA000B6180022307830277F423F18FFB2092F36
:102AB00007D80A277A438218D2B2303AD2B2013606
:102AC000F0E7AF18BC46029FBC4501D97A1BD2B2D1
:102AD000692818D00BD863282AD0642813D0582826
:102AE00032D11F1D1B68201C009301231DE0752897
:102AF0000FD0782814D0732826D11F1D201C1B68E6
:102B0000FFF708FF0AE01F1D201C1B68FFF73FFFAF
:102B100004E01F1D201C1B68FFF713FF3B1C0BE08C
:102B20001F1D1B68201C00930023FFF769FFF5E7BA
:102B30001868043320700120721C24182D188BE7AC
:102B4000013C2370681E01E00120404205B0F0BD49
:102B500010B50C1C131C6421221CFFF775FF10BD5F
:102B600000B5031C9BB00A1C01A8191CFFF7F0FF5D
:102B7000632800DDFEE701A800F0B6F81BB000BD39
:102B80000FB407B504A908C9181C0191FFF7E8FFA5
:102B900003B008BC04B018470EB403B503AA08CAB2
:102BA000191C0192FFF7D4FF02B008BC03B018470C
:102BB00030B50C1C044303232340041C002B01D01C
:102BC000002310E0032AFBD9CC58C4500433D41A94
:102BD000032CF9D8131F9B0801339B00C418C91894
:102BE00003231A40ECE7934203D0CD5CE554013354
:102BF000F9E730BD30B5031C840701D1032A01D8A1
:102C00009A1814E00B060C041D1C25430D430C02FE
:102C10002543031C20C38418E41A032CFAD8131F7D
:102C20009B0801339B000324C3182240E8E793422A
:102C300002D019700133FAE730BD021C031C981A48
:102C40000133591E09780029F9D17047031C0A780D
:102C50001A70002A02D001310133F8E7704730B50D
:102C60000023934208D0C45CCD5C651B06D10133C0
:102C7000002CF6D1201C02E0002000E0281C30BD12
:102C800010B50022835C8C5CA34204D10132002B7E
:102C9000F8D1181C00E0181B10BD000008B5094B46
:102CA000FA211868890002F0D1FAFFF731FB96206B
:102CB0000002FFF77DFD0120FDF7C4FAFEF742FF99
:102CC00008BDC0469804001008B5FEF7C3FFFFF723
:102CD000F9F8FFF7A1F9FEF781FBFEF76DFBFFF7AF
:102CE000DDFFFFF7E7F808BD10B5041C20780028C9
:102CF00003D00134FDF7F6FAF8E710BD38B5051C2E
:102D00000E24013C04D3295D0248FFF739FFF8E7A0
:102D100038BDC046705F000038B51948FFF730FF76
:102D2000184C201CFFF7EAFF174D4221281CFFF723
:102D300027FF201C0E30FFF7E1FF4321281CFFF77F
:102D40001FFF201C1C30FFF7D9FF1048FFF718FFAA
:102D5000201C4630FFF7D2FF0D48FFF711FF201C63
:102D60002A30FFF7CBFF281C4E21FFF709FF201C5C
:102D70003830FFF7C3FF616D0648FFF701FF38BD2C
:102D8000735F0000D4040010795F0000805F0000D2
:102D9000865F00008C5F000003110A2253430F225C
:102DA00010401818704738B50A21041C02F04EFA7A
:102DB0000A210501201C02F09FFA281C084338BD97
:102DC00008B5C12252000E200221FEF715FE024B6B
:102DD00001225A7108BDC046C804001010B5084C45
:102DE0006379002B01D1FFF7EBFF23790C221A4303
:102DF000A37901205B001A43011CFEF7FDFD10BD05
:102E0000C804001010B5074C2379002B08D1637952
:102E1000002B01D1FFF7D4FF01232371FFF7DEFF61
:102E200010BDC046C804001008B5054B1A79002A29
:102E300005D000221A711A72DA70FFF7CFFF08BDB1
:102E4000C804001010B501210220FEF713FE064B46
:102E5000041C18787F231840FFF79EFF034B58701F
:102E6000DC71201C10BDC046A4040010C804001072
:102E7000014B01229A707047C8040010024B0022D7
:102E80009A701A727047C046C804001008B5FFF760
:102E9000D9FF094B094A9978002908D0197A0129E4
:102EA00001D8013103E010680549086000E019729B
:102EB0000021D970116008BDC80400106C02001018
:102EC0007002001008B5FEF71BFE0C23184003D05B
:102ED000024B1A781043187008BDC046C804001091
:102EE00010B5FFF7EFFF054B1A781C1C530701D5EF
:102EF000FFF7CCFF0023237010BDC046C8040010AC
:102F000008B50020FEF7E2FB002801D0FFF7E8FF3C
:102F100008BD000010B5054C0023E371FFF7F0FF7A
:102F2000E379002B01D1FFF78DFF10BDC80400101D
:102F300008B50948092102F0EBF9084BFA22D20042
:102F40001A80FFF7E7FF064B00221A60FA22054BB2
:102F500092001A6008BDC046C8040010D2040010D8
:102F60006C0200107002001008B5FFF7C9FF0020C6
:102F700008BD08B5FFF758FF08BD000070B51D4C2F
:102F8000061C637822781B021343A278A0791204EE
:102F90001343E2780D1C12061343174A13401A0A12
:102FA000237062701A0C1B0EE3706379A270227991
:102FB0001B021343114A134023711B0A6371FFF76D
:102FC000EBFE0F4B1B88C01830806079FFF7E4FEE2
:102FD000B070E078FFF7E0FEF070A078FFF7DCFE5D
:102FE00028706078FFF7D8FE68702078FFF7D4FE6D
:102FF000A87070BDA40400107F7F3F3F071F000032
:10300000D2040010F0B58DB0051CFEF743FD00287A
:1030100004D1281C1249FFF7BFFD1EE00AAE0BAC1D
:10302000211C301CFFF7AAFF3388F7780793B37889
:10303000267808936378A47809930A4B187900F0EE
:10304000D7F8099B04900293009701960394281CDB
:103050000549079A089BFFF79FFD0DB0F0BDC046DC
:10306000985F0000A40400109D5F000070B5061C6E
:103070000D1C141CFEF70EFD00280AD0301C291C64
:10308000FFF77CFF002C07D0044B00201B79236046
:1030900003E00120404200E0201C70BDA4040010A9
:1030A000F7B504880E1C051C6421201C00920193B6
:1030B00002F0C2F8114B8FB2B078E41B1C80FFF70E
:1030C00072FE0F4CA0707078FFF76DFEE0703078E4
:1030D000FFF769FE2071E878FFF765FE009B6071DD
:1030E000A371A878FFF75FFEE071381CFFF75BFE65
:1030F00020720198FEF7E0FCFEBDC046D20400102D
:10310000B404001008B50223FFF7CAFF08BD08B5D4
:10311000021C501E8241520100200121FEF76CFC6E
:1031200008BD38B5041C01200D1CFFF7F0FF201C62
:1031300000F086F8072102F0DFF8201C0A1C291C89
:10314000FFF7E0FF96204000FFF7FCF80020FFF7B4
:10315000DEFF38BD73B5041CFFF774FE002801D1F3
:1031600000203BE01E4B5D781E1C7378AB4207D1FC
:103170000A20FFF7E7F8FFF765FE0028F5D1EFE733
:10318000FEF788FC0028EBD001A96846FFF7F6FEA1
:10319000684600F055F8051C01A800F031F8114B05
:1031A00004199C420DD9E31701221343ED18281C82
:1031B000694600F075F8002C01DA0B4B00E00B4B70
:1031C000E418201C01A900F024F8281C072102F0B3
:1031D00093F868460A1C01A9FFF794FF76BDC04624
:1031E000C80400107F5101008051010080AEFEFF35
:1031F00007231840014B8000C05870471060000042
:1032000002783C235A4341785218534382789818E5
:10321000704738B50C1C3C21051C02F06DF8281CC9
:10322000A1703C2102F012F83C2102F065F86170B7
:10323000E121281C090102F009F8207038BD0000C6
:1032400070B5837802210022994252410488962168
:103250004901051C64180C20A41A42439B18033B27
:10326000992058430521023001F0F0FF6E26FF3609
:1032700066436421A31086194942201CF61801F008
:10328000E5FFC82136184900201C01F0DFFF034B81
:103290003018C018EB78C01870BDC046D382FFFF4D
:1032A000F8B5204B0C1CC5181F4B8000C0181F49D7
:1032B00001F0CCFF03235843C617B60F3618B610DB
:1032C000AE19B600953E301C194902F015F8CD171D
:1032D000AD0F6D180527AD107D430235281C9921CF
:1032E00002F00AF8081C391C01F0B0FF0130E07050
:1032F0009921281C01F0AAFF0C21023001F0FCFFEB
:103300004D1CEDB2A570301C094901F09FFF094B1F
:103310000C21C6180E20401B01F098FF361826809D
:10332000F8BDC04679050000652F0400B13A0200DF
:10333000B505000094EDFFFFF8238A01DB00134080
:103340004A05920E1343F8221202114019430A2330
:10335000594330B5CA1083181C1CEB345D782478AF
:10336000EA336C401B7824021C43835C201C5840C9
:103370000723194008418005800D30BD70470000CB
:1033800008B5054B011E994201DD044BC1180448E4
:10339000EA38FFF7D1FF08BDFF17000000F8FFFF74
:1033A0004C6000000723594310B5084B59189C3155
:1033B0000023CC5C0F2222400270CA5C0133120948
:1033C00042700230072BF4D110BDC046D404001067
:1033D0000723594310B5074B59189C3100234278F5
:1033E000047812012243CA5401330230072BF6D16C
:1033F00010BDC046D404001070B5AD4C86B0E36E6D
:103400006E465A1E934117363370AA4B9A6A191C9E
:10341000D006400F0138062807D801F0B5FE040C8D
:103420002012181A1D00022509E0636E16339B0056
:103430001B591D1C15E0636E16339B00E5580023D5
:103440000FE0A36DE56DAB420BDD0D2509E0022514
:1034500003E00C25032304E00D252B1C01E00D25C2
:10346000EDE70D6150111F2800D91BE101F096FE18
:103470002000220029002C002F0033003B004400D4
:1034800048004C00540061006E00760083008F00FD
:103490009B00A800B800C500D500D300E100E400FF
:1034A000E700EF00FE0002010B010D010F01150105
:1034B000E01801E0E0180E30EB1A591C01F028FF6B
:1034C000F0E0E0181C30F7E7211C0E3105E0E018B1
:1034D0000E30E1180BE0211C1C31201C1A1C2B1C87
:1034E00001F095F9DEE0E018E1181C300E31EB1A1E
:1034F0005A1CFFF75DFBD5E06F48011C0E31EDE76C
:10350000E018011C1C31F2E7226E1021002A00D0C5
:103510000A21221C0E3206E0226E1021002A00D061
:103520000A21221C1C32029100950196201C211CAC
:1035300053E0216E012232701022002900D00A22AD
:10354000009501960292201C211C45E0226E10215C
:10355000002A00D00A21221C0E3213E0216E012223
:1035600032701022002900D00A22009501960292A2
:10357000201C211C4DE0226E1021002A00D00A21BF
:10358000221C1C32009501960291201C6AE0226EDA
:103590001021002A00D00A21484A02910095019684
:1035A000101C111C19E0216E1020002900D00A20E7
:1035B000424A0290111C1C3900950196101C0CE027
:1035C000216E012232701022002900D00A223B49CC
:1035D000009501960292081C002201F022F961E098
:1035E000226E1020002A00D00A20344A0290111CBA
:1035F0001C3900950196101C35E0216E01223270B5
:103600001022002900D00A222C490095019602922E
:10361000081C002227E001223270226E1021002AAD
:1036200000D00A21254A029100950196101C002124
:1036300019E0009620481BE00096204818E0226E12
:103640001021002A00D00A21221C1C3206E0226E22
:103650001021002A00D00A21221C0E32009501966A
:1036600002910020211C01F004F91BE00096201CAF
:10367000002103E0211C1C310096201C1A1C2B1C6D
:1036800001F05AF90EE0201C02E00B4800E00B4864
:10369000191C2A1C01F067F904E0201C191C2A1CC3
:1036A00001F06BF933780120E36606B070BDC046C7
:1036B000D4040010700C0010E2040010F00400109C
:1036C000064910B50A1C883213681C1C1E34A4005D
:1036D0006050013303210B40136010BDD40400106F
:1036E000054B0322191C88310868013802400A6022
:1036F0001E329200D0587047D4040010F7B5124F14
:103700003D1C8C3528680130FFF73AFE0F4EBB6E2A
:10371000B26A041C01920122F06202409A4210D166
:10372000830703D428680230FFF7CAFFFF239B00FA
:10373000019A1C40A40193101C438C3701233C6068
:10374000F3600220FEBDC046D4040010700C0010CF
:103750000C490D488A6A031C8C3370B51D68D3056B
:103760009B0E0C1C910500D5403B866E92100121EA
:103770000A40B24203D18C30EB180360E1600120B3
:1037800070BDC046700C0010D404001008B5084B82
:103790005A1CD07F9A1CD27F0001120210430333BF
:1037A0001A7FDB7F10431B031843FFF789FF08BD17
:1037B000D404001008B5FFF793FF0323044A0F2138
:1037C0009A180140013311770011072BF6D108BD7B
:1037D000D404001008B5FFF783FF034B01228C339C
:1037E0001860024BDA6008BDD4040010700C0010A1
:1037F00010B5064CA36E002B06D0FFF771FF044BEB
:103800008C3401222060DA6010BDC046D404001060
:10381000700C001010B5064CA36E002B06D1FFF7FC
:103820005FFF044B8C3401222060DA6010BDC0467B
:10383000D4040010700C001008B5044B01221A6269
:10384000034B1B68002B00D0984708BD700C00107C
:103850003403001008B5104B0022596A1A629142D5
:1038600014D05969914216DD012906D1D9699142D6
:1038700003D0DA610A2299615A615A69032A02DD8A
:1038800006490120C866013A5A6104E0044B1B68EE
:10389000002B00D0984708BD700C0010D404001015
:1038A00034030010074B5A6A002A02D05A69002AD2
:1038B00007DD9A690F21044B1140D97712110133AA
:1038C000DA777047700C0010D4040010044B597F55
:1038D0009A7F090112020A43197F0A435A67704707
:1038E000D40400100B1C093B10B5012B0FD800238A
:1038F000074A9A18147FC25C944205D0054B0839D8
:103900005A681143596002E001330E2BF0D110BD0B
:10391000D4040010700C001008B508290DD0192926
:1039200013D1427808231A4202D00022027002E02A
:103930000F2303700723437005E000230022C254C5
:1039400001330E2BFAD1FFF743FD08BD30B5114D01
:1039500085B06C6F002802D00F239C4304436C6732
:10396000FF2C05DD281C1C300E2101F0D1FC0FE0DE
:103970006846211CFFF716FD6846211CFFF7CCFFA7
:1039800000236846C15CEA18013311770E2BF8D189
:1039900005B030BDD4040010134B30B5596F0F2261
:1039A0009143041C0C4385B05C671D1C082C19D086
:1039B000FF2C17DC6846211CFFF7F4FC6846211C2D
:1039C000FFF790FF0023EA18127F6946CA540133BB
:1039D0000E2BF8D16846211CFFF79EFF6846211C7C
:1039E000FFF7F6FC05B030BDD40400101FB50F4C36
:1039F000616F082918D0FF2916DC6846FFF7D2FC52
:103A00006846616FFFF76EFF0023E218127F694678
:103A1000CA5401330E2BF8D16846616FFFF77CFF63
:103A2000616F6846FFF7D4FC1FBDC046D404001088
:103A300010B50D4C631CD87FA31CDB7F00011B025B
:103A40001843E37F1843E31CDB7F1B031843FFF796
:103A500097FC0F23021C1A40227702111340001218
:103A60006377A07710BDC046D4040010044B5A6E93
:103A700016329200D258121A51424A41DA66704701
:103A8000D4040010044B5A6E16329200D1580139FA
:103A900000D50D21D1507047D4040010054B5A6E4B
:103AA00016329200D15801310E2900D10021D15097
:103AB0007047C046D4040010094B5A6E163292006B
:103AC000D2580D2A03D11A1C2932127805E09A180F
:103AD000507F117F0001021C0A435A657047C0469F
:103AE000D4040010084B10B55A6E0F241632920001
:103AF000D1585A6D58181440013104770D2902DC51
:103B00005B1812111A7710BDD40400100E4B30B59B
:103B10005A6E596D16329200D2580D2A07D11C1CCC
:103B20002934F020247808402043586507E098188D
:103B3000447F057F24012C435C650C1144779B185E
:103B40000F221140197730BDD404001008B5034886
:103B50000E22011C1C39FFF72BF808BD0C050010C4
:103B600008B503480E22011C1C31FFF721F808BDDF
:103B7000F004001008B504480022011C1C310D237C
:103B800000F045FE08BDC046F004001008B503482B
:103B90000E22011C0E39FFF70BF808BDFE040010C1
:103BA00008B503480E22011C0E31FFF701F808BDCD
:103BB000F004001008B504480022011C0E310D234A
:103BC00000F025FE08BDC046F00400100023044AA2
:103BD00000219A18463201331170082BF7D1704733
:103BE000D4040010C31C421E0020934207D0044995
:103BF0004000591846310978013B0843F5E7704702
:103C0000D404001010B50B1D994208D0044A0124B9
:103C10008A1804404632147040100131F4E710BD98
:103C2000D404001038B50020FFF7DCFF084C051C59
:103C30000021207FFFF7E6FF04202577FFF7D2FF62
:103C40000421051C607FFFF7DDFF657738BDC046A6
:103C5000D404001010B50020FFF7C4FF034C2077F8
:103C60000420FFF7BFFF607710BDC046D4040010EA
:103C700010B5054C0021207FFFF7C4FF607F0421B1
:103C8000FFF7C0FF10BDC046D404001010B5094CAA
:103C9000231C8C3318680130FFF772FB064B021CA3
:103CA000D8620F231A402277021113400012637763
:103CB000A07710BDD4040010700C001010B5084C93
:103CC0000E21201C01F024FB201C0E300E2101F0DF
:103CD0001FFB201C1C300E2101F01AFB10BDC0463A
:103CE000D404001010B50C4B191C0E311A1C187F8F
:103CF0001C7801332043D8768B42F8D1936E002B89
:103D000008D0064B1B690D2B04D1137F111C2931E0
:103D10000B70537310BDC046D4040010700C00101B
:103D200010B50C4B191C0E311A1C1C7F187801336E
:103D30002040D8768B42F8D1936E002B08D0064BEA
:103D40001B690D2B04D1137F111C29310B70537388
:103D500010BDC046D4040010700C001030B5002116
:103D600085B00E4B421C1818007F6C4608550D2577
:103D7000D40F181C002395425C416442013122405B
:103D80000E2901D0101CECE76C46E15CC21801332F
:103D900011770E2BF8D105B030BDC046D404001009
:103DA000074B10B55A6E16329200D458611E1C197A
:103DB000D1502077002901DA0D21D15010BDC04625
:103DC000D4040010034A0023111C943198320B6074
:103DD00013607047D4040010034B01229433196818
:103DE0004A401A607047C046D4040010044A0023B9
:103DF00013678C321360034B0122DA607047C046B0
:103E0000D4040010700C001008B59E4B0F20996A66
:103E10009D4A8B1018408911013852560E2848D8F7
:103E200001F0B2F9080F171F2347294747314747C9
:103E300047353900002A3CDB944B9A184032002366
:103E400005E0002A35DB914B9A184032012393712B
:103E50002DE0002A2DDB8D4B9A1840329279DA66DC
:103E600025E0081CFFF79CFF21E0002A21DB101C45
:103E7000FFF7FCFD1BE0002A1BDB844B596E16315B
:103E80008900CA5013E0081CFFF786FD0FE0081CEC
:103E9000FFF75CFD0BE0002A0BDB101CFFF75EFF59
:103EA00005E00C2B23DD162B28D1FFF705FE0120A2
:103EB000EEE0982B03D1754B00221A66F7E7982B9A
:103EC0006CDC382B03D1714B01205866E0E0382BB5
:103ED00030DC1C2B02D1FFF739FEE8E71C2B12DC8B
:103EE0000C2BDED1694B012098331860D0E0012003
:103EF000002B00D1CCE001204042C9E0182BFAD1C0
:103F0000FFF774FFD3E7282B03D1604B00225A66DA
:103F1000CDE7282B04DC262BEDD1FFF7E3FDC6E728
:103F20002C2B02D1FFF71CFEC1E7362BE3D1FFF7A4
:103F3000EDFDBCE7662B02D1FFF732FEB7E7662B3B
:103F400016DC4C2B03D1FFF7A1FE0220A0E04C2B86
:103F500004DC3C2BCFD1FFF70DFEA8E7562B02D196
:103F6000FFF714FEA3E75C2BC5D1FFF70FFC9EE71C
:103F70006C2B02D1FFF71EFC99E76C2B04DC682B3D
:103F8000B9D1FFF79BFE92E7762B02D1FFF712FE25
:103F90008DE7882BAFD1FFF785FC88E7E62B02D1B0
:103FA000FFF758FE83E7E62B35DCC82B02D1FFF77D
:103FB00013FF7CE7C82B16DCA82B03D1334B012061
:103FC000186665E0A82B04DC9C2B94D1FFF77EFCDF
:103FD0006DE7B82B02D1FFF7F5FE68E7BC2B8AD15D
:103FE000FFF704FD63E7D62B02D1FFF741FE5EE742
:103FF000D62B05DCCC2B00D07DE7FFF719FD56E76B
:10400000D82B02D1FFF7F4FB51E7DC2B00D072E78D
:10401000FFF768FE4BE7F32B02D1FFF71BFC46E7E7
:10402000F32B17DCEC2B02D1FFF77AFE3FE7EC2BEA
:1040300005DCE82B00D05EE7FFF7ECFB37E7F12B60
:1040400002D1FFF7C3FD32E7F22B00D053E7FFF7B1
:10405000F3FB2CE7F62B02D1FFF7E4FD27E7F62B65
:1040600005DCF52B00D046E7FFF70CFD1FE7F72B2B
:1040700002D1FFF713FD1AE7F82B00D03BE7FFF75B
:10408000A9FB14E7700C00104C9C0000D404001035
:1040900008BDC04638B5184C231C8C331868FFF790
:1040A0006FF9164B0022E16EDA60E2660322986235
:1040B000A16610401D1C022809D090420AD0012898
:1040C00002D0FFF7A1FE07E0FFF718FB04E0FFF7BF
:1040D00093F901E0FFF73CFB00280BDDEB68002BB8
:1040E00004D1231C8C3319680A181A609034226892
:1040F0001318236038BDC046D4040010700C0010A3
:10410000034B0122DA660F229A775A771A777047A3
:10411000D404001010B5054C0549201C01F0F8F836
:10412000FFF7EEFF0123636610BDC046D404001004
:104130009C0700007047000030B50C4D049C2860BF
:104140000B4801600B490A600B4A13600B4B039A42
:104150001A600B4B0B4A1C600B4B1C600B4B1A601C
:104160000B4B0C4A13600C4A136030BD6003001007
:10417000700300107C030010440300103C03001087
:1041800010000010A9420000700C00103403001051
:10419000354100007403001058030010014B1860F3
:1041A0007047C04640030010094B10B51A68191C2F
:1041B000084B002A03D1084C2468226003E01A68E7
:1041C000904200DA101C186001230B6010BDC0463D
:1041D000480300106C03001040030010034B1B68E1
:1041E000002B01D1024A13607047C04654030010EF
:1041F00048030010014B4A3318787047D40400106C
:1042000038B5164B1A1C98321268002A04D0144B89
:104210001C6801231C4001E094331C68114DAB68FD
:104220009C4202D16A68002A16D0002C02D1002BD1
:104230000AD111E00C4B1B68002B02D0201C6968CE
:10424000984700236B6006E0074B1B68002B02D0E9
:10425000201C211C9847AC6038BDC046D404001017
:1042600050030010700C001060030010084B186021
:10427000084B1960002809D0074A01231370074A28
:1042800000211170064A9061064A13707047C046BB
:104290005C03001078030010640300104C0300104E
:1042A000700C0010380300102D4B73B51A682D4B9D
:1042B0001168186881421BD0002100910191126899
:1042C0001A60294B1B688B4202D0684601A99847A7
:1042D000264B00991C68181C019A254BA14202D15B
:1042E0001C68A24202D0234C0125257001601A608F
:1042F000214E336A002B10D01E490023CB56002BD1
:104300002CD01E4B00229A56012A27D100220A7077
:104310001B490A7002221A7020E0144B174C1868CF
:10432000002807D00023E356002B03D1104B196857
:10433000FFF79CFF0023E356114D022B03D100230E
:104340002B70B36123700023E356002B02D00A20A8
:10435000FFF72AFF0022AA560A4BDA6673BDC04651
:10436000440300100C000010700300105C030010E8
:10437000780300104C030010700C0010380300107C
:1043800064030010D404001008B5084A084B1268F2
:1043900019688A1A05D5FA2252001A60054B1A6864
:1043A00001321A60FFF72CFF08BDC0463C03001025
:1043B0001400001050030010F8B50E1C0E21041C50
:1043C000171C00F0A5FF174B03259E4211DD0923A2
:1043D00063730123237323E0301C0A2100F08CFF58
:1043E000301C61550A2100F031FF0135061C0D2DEE
:1043F00001D0002EF0D1EF1B033F27706B1E022B64
:1044000005D0E15C621BD2185173013BF7E70F2323
:104410005D1B013D6B1C032B02DD00236355F8E798
:10442000F8BDC046FFC99A3B37B5041C00250023E0
:1044300000930193124B1B68002B02D0684601A920
:10444000984700980135002800D000250220FBF78E
:10445000A5FF0C4B1A680C4B1168186881420AD0F2
:1044600012681A60FFF790FF002C04D0013C002C6A
:1044700001D1201C02E0032DD9DD01203EBDC04644
:104480007003001044030010680300100278002A33
:1044900001D1802252004378002B01D180235B00A0
:1044A000D01A7047F0B59B23234D5B00EC5C85B0C0
:1044B00003900E1C002C01D1802464003023FF33B4
:1044C000EB5C002B01D180235B0002933823FF3388
:1044D000EA5C80235B009C4203D00F23171C1F4023
:1044E00000E007271548FFF7D1FF0299421C631A25
:1044F000802149000C1B0721C91B009401910398DE
:104500000F49FEF749FB002333704124301CFEF7AE
:1045100094FBBA235B003718E818001BFFF7B6FFBF
:10452000221C031C0749381C0134FEF735FB462CBE
:10453000ECD105B0F0BDC046D40400100806001050
:104540005C9C0000699C0000F0B5634D634C2B1C23
:1045500094331B6893B0061C0F1CA061E161002B13
:1045600017D118280BD1C32909D15D4B1B680F2B1C
:1045700005D1281C38300E21162200F033F9A0692D
:10458000182804D1E269332A01D100F0D1F8FFF7ED
:10459000B7FD002E02D00A23636100E06661301C83
:1045A000391CFFF763FE4F4E33681A684E4B1A6092
:1045B000FFF714FE01232B670020142300930190C2
:1045C0004A4B1B68002B1AD0494E3368371C002B0E
:1045D00015D01B68002B04D1464B1B6898473B68DD
:1045E000F7E733681A68013A1A60434A1368002BE8
:1045F00005DD013B1360002B01D1FFF7EFFDFFF755
:1046000049FD002801DAFBF785FF3C4B019A9A42ED
:1046100004D040239A433A4B9A420BD1A36A394AB9
:10462000934204D008229343374A934202D10A208E
:10463000FFF7BAFDA36A2E1C8C360193334A336808
:1046400093421AD0324A93420FD0324A934223D136
:10465000FFF7D6FDFBF7D2FE2F4BA0611860224B6F
:104660001A68013A1A602D4B15E02D4B1B68002B80
:1046700012D00120616898470EE02A4F3868002860
:104680000AD002A80AA9FFF70DFF3B6802A80AA9F1
:104690009847336827333360009E009A013E002A12
:1046A00003DC214B14261B6898470E4B1A681F4BDE
:1046B00011681868814206D012681A60FFF764FE1C
:1046C0000C4B1B6898472A6F002A01D0009677E7A9
:1046D000FFF796FD13B0F0BDD4040010700C00106D
:1046E00010000010440300100C00001048030010DC
:1046F00040030010740300106C0300106E020000F1
:1047000026020000FB030000E30300003E27000038
:104710005C280000790D00005C0300107E0D000095
:10472000600300107C0300105803001068030010A1
:10473000F7B5274E002033681C68FFF775FE336815
:104740001A689442FCD01B6801272D33FF33019374
:10475000FFF7D6FC1F4C0A231F4D63611823A3618A
:104760001523E3612B1C9033002267621A60FFF768
:10477000C7FC2F673368019A1B689A420CD0FFF779
:1047800089FC3268154B116818688142F2D01268B2
:104790001A60FFF7F9FDEDE72B1C01279033182075
:1047A00000211E686762FFF7CFFE0D4B301C1968B1
:1047B00000F04CFD3835011C0422281CFFF7FCFDDD
:1047C0001823A3610023301C6762E361FEBDC0466D
:1047D00044030010700C0010D40400106803001093
:1047E0003C03001070B5002A10DD047801231C4042
:1047F0004B1E002B08DBC55CE4006E083443C45438
:104800000124013B2C40F4E7013AECE770BD30B5E0
:104810009A4205DC845C8D5C85548C540132F7E748
:1048200030BDF0B5069E051C07A804783078002A34
:1048300017D0059EB34217DCCE5CD75CF7193F1842
:104840000020A74201DB3F1B0120EF540133F0E7BA
:10485000CA5C12180020A24201DB121B0120EA549C
:104860000133059A9342F3DD01231840069B18702B
:10487000F0BDF7B50AAC2478099D0094089E2C7809
:10488000002833D000292ED0002A1CD0B3424EDCA1
:10489000CF5CD55C7F1B3F1B0024A74204DA009C41
:1048A0003F190F2427400124C7540133EEE7CA5CA7
:1048B000121B0024551C04D1009C0F22013C2240F5
:1048C0000124C2540133B342F1DD30E0D15C4942EE
:1048D000091B0024A14204D0009F0F24C9192140C4
:1048E0000124C1540133B342F0DD20E0002914D08B
:1048F000002A08D0B3421ADCCD5CD05C0133281A00
:10490000041BE40FF6E7B34211DCCA5C0133141B4D
:10491000013462425441E4B2F5E7B34207DCD15CB2
:10492000013349420C1B611E8C41E4B2F5E70123BF
:104930001C40099B1C70F7BD70B5049C01252570B7
:1049400000290BD09A420BDC865C8D5CAE4209D10B
:104950000132F7E7815C002904D101329A42F9DD86
:104960000023237070BD914204DA43185B784354EE
:104970000131F8E70023435470478A4205DD83186C
:10498000013B1B788354013AF7E7002383547047B7
:10499000F7B5134A134C13785278C35C134000D018
:1049A0004023114923601231009100220023A618F0
:1049B0007360009B0125123B1F785978C75D39420F
:1049C00002D077682F437760009F02336D00BB42AF
:1049D000F2D1123304320093282AE7D10020FEBD21
:1049E00004010010300E001050000010122330B5EA
:1049F0004B43334A0131D318052251431A785C786E
:104A0000825C144204D02F4A5F2452189470547070
:104A10009A78DC78825C144204D02A4A7C245218AA
:104A2000533214701A795C79825C144204D0254A9E
:104A30007C245218A33214709A79DC79825C144277
:104A400007D0204C5F226418251CA235A1342A709F
:104A500022701A7A5C7A825C144204D0194A7C244F
:104A60005218A03214709A7ADC7A825C144204D014
:104A7000144A7C245218503214701A7B5C7B825C7E
:104A8000144207D00F4C5F226418251C5235513454
:104A90002A7022709A7BDC7B825C144204D0094A23
:104AA0002E245218A43214701A7C5B7C825C134250
:104AB00004D0044B5918F43127230B70002030BD6B
:104AC00050000010A00C0010F8B52E4D061C002759
:104AD0002C1C281C20214F22FEF78CF8002F04D01C
:104AE0002A1C7C2339322B7013702B1C4F3300226D
:104AF00001371A705035052FEBD1211C2D23383189
:104B00000B70211C37310B70A121A3706370490019
:104B10005F2363544221FF316354A321490062544F
:104B2000194A11785278715C0A4204D0221C53321F
:104B30005234137023700024211C301C0134FFF701
:104B400055FF0A2CF8D10024104B114DE25C1B19C3
:104B5000B15C58780F4A6300084201D0D15805E093
:104B6000D058FEF76AF80C49091A0A31281C023499
:104B700000F0D8FB122CE7D1281C084900F0D2FB2A
:104B80000520F8BDA00C0010040100101800001052
:104B9000E00D00102C00001006010010719C0000B8
:104BA000F0B5944B87B003901F68FCF705FC924961
:104BB0000022924C02910192019B0C255D43002B37
:104BC00000D101258B4B1968032903D0042900D19A
:104BD0003EE202E0884A029202E0022900DCAAE0FA
:104BE000002305AA537023687F2003405B2B72D0FB
:104BF0002CDC232B00D19AE014DC062B50D006DCF1
:104C0000002B4BD0022B00D094E0492390E01C2BCA
:104C100000D18AE0212B00D185E0072B00D089E06C
:104C2000372385E0402B6ED008DC392B6FD03F2B2B
:104C300067D0382B00D07DE04C2379E0502B72D028
:104C4000542B74D04F2B75D1332371E0732B68D064
:104C500012DC662B41D007DC5E2B5AD0622B64D06D
:104C60005C2B67D14F2363E06F2B3CD0712B54D06A
:104C70006D2B5FD135235BE0792B4CD006DC762B96
:104C80004DD0772B41D0742B54D148E07D2B26D0CA
:104C90007F2B26D07C2B4DD1422349E0202347E0B7
:104CA00031231370019B022B00DCB8E1231C083B6D
:104CB0001B680340542B0AD00199032900D1AEE1AF
:104CC000231C0C3B1B681840542800D0A7E14C2241
:104CD00005AB1A70A3E132232AE0342328E03623FF
:104CE00026E0382324E039231370019B062B00DCD7
:104CF00095E1231F1B6818404723232800D08EE12D
:104D000016E0302314E02D2312E0412310E043236A
:104D10000EE044230CE045230AE0462308E0482344
:104D200006E0502304E0522302E0552300E04E2326
:104D3000137074E1CF1E012F62D0022F00D1E1E089
:104D4000002F00D03EE1226801231A4205D0A81CA2
:104D5000C0B2391C0522FCF7A7FB23689B0706D5C8
:104D6000E81D0121C0B20A1C0323FCF79DFB21684A
:104D70000423194205D0E81DC0B205210122FCF729
:104D800093FB2268120706D5A81CC0B20921052290
:104D90000123FCF789FB2368DB0606D5681CC0B23B
:104DA000052101220423FCF77FFB2168890606D533
:104DB000681C0121C0B20A1C0323FCF775FB2268A2
:104DC000520606D5A81CC0B2042105220123FCF717
:104DD0006BFB23681B0607D5281C0930C0B20921CC
:104DE00002220123FCF760FB2168C90500D4E9E039
:104DF000DCE0C04614010010B45C0000300E00106E
:104E000022683A420ED0EEB2B01CC0B20021052298
:104E10003B1C0336FCF748FBF0B2391C03223B1C59
:104E2000FCF742FB23680222134205D0A81DC0B242
:104E300001210323FCF738FB21680423194205D024
:104E4000A81DC0B205210222FCF72EFB226808260D
:104E5000324211D0EBB2181C02300093C0B20921CB
:104E600005220123FCF720FB009B311C0333D8B241
:104E700003220123FCF718FB2168C90606D5681C2C
:104E8000C0B2052102220423FCF70EFB2268920621
:104E900006D5681CC0B2012102220323FCF704FBE3
:104EA00023685B060ED5EEB2B01CC0B20421052209
:104EB00001230336FCF7F8FAF0B20521032201239F
:104EC000FCF7F2FA2168090607D5281C09300222EE
:104ED000C0B20821131CFCF7E7FA2268D20571D58D
:104EE000EDB22E1C0A36F6B2301C08210222032332
:104EF000FCF7DAFA0935301C0B21FCF7C1FAE8B2ED
:104F00000B215DE02368DB0706D5681CC0B20021D9
:104F100007223B1CFCF7C8FA21680222114205D087
:104F2000A81DC0B200210623FCF7BEFA22680421A6
:104F30000A4205D0A81DC0B202220623FCF7B4FA2B
:104F4000236808210B4205D0681CC0B20722022347
:104F5000FCF7AAFA2168C90606D5681CC0B204216C
:104F600002220623FCF7A0FA2268920606D5681CE6
:104F7000C0B2002102220623FCF796FA23685B06E2
:104F800006D5681CC0B2042107220223FCF78CFA64
:104F90002168090607D5281C09300222C0B2082161
:104FA000131CFCF781FA2268D2050BD5EDB2281C40
:104FB0000930C0B20B210A35FCF762FAE8B20A21C7
:104FC000FCF75EFA019B0434013301930B2B00D0F4
:104FD000F2E5214B1B68002B05D020480021092257
:104FE0001F4BFCF7D7FA1F4D00240235AB1E1A7871
:104FF00003996B1E8A5C1B78134208D01A4BA200DF
:10500000D0581A4B0922E15C154BFCF7C3FA013466
:105010000235092CEAD1FCF7D9F907B0F0BD00221E
:1050200005A8291C029BFCF7B5FA2268120605D5D3
:10503000E91D0F480022029BFCF7ACFA2168C90564
:10504000C0D5E91D0B480022029BFCF7A3FAB9E783
:10505000094B0293C4E5C0464C0100107B9C000044
:10506000AC5C00001800001018010010D49C000077
:105070009D5D0000799C0000BC5C000038B5FFF726
:10508000B9F80624002805D1FCF7A0F938BD013491
:105090000E2CF9DC0321201C00F0D8F80321C5B246
:1050A000201C00F029F9281CC9B2FCF7E9F9092CE9
:1050B000EDD10B24EEE7000038B5041CFFF768FCC7
:1050C000201CFFF76DFD094B1B78002B0DD0201C19
:1050D000FFF7FAFC064CC8235B00E518211C0548C5
:1050E0005034FDF74DFDAC42F8D138BD89030010B6
:1050F000A00C0010B254000000B589B000280ED0FA
:10510000FCF725F901A80921FEF74CF96846123091
:105110000A21FEF747F901A8FFF7CEFF08E0FCF7E8
:105120001EF9044B1B78002B02D00348FDF728FD25
:1051300009B000BD890300107D9C0000FEE7FEE77A
:1051400008B500230B4A0C499A188A4204D20B492D
:10515000C95C01331170F5E7094B0A4A591C013B40
:10516000934203D200221A700B1CF6E7FBF79AFD5C
:10517000FEE7C046000000103C010010DD9C00006E
:105180003D0100105C0E001002B471464908490050
:10519000095C49008E4402BC7047C04603B47146A6
:1051A000490840004900095A49008E4403BC704731
:1051B000002934D00123002210B488422CD30124CA
:1051C0002407A14204D2814202D209011B01F8E75F
:1051D000E400A14204D2814202D249005B00F8E718
:1051E000884201D3401A1A434C08A04202D3001B44
:1051F0005C0822438C08A04202D3001B9C08224377
:10520000CC08A04202D3001BDC082243002803D0B4
:105210001B0901D00909E3E7101C10BC70470028E6
:1052200001D00020C04307B4024802A140180290F8
:1052300003BDC046D90000000029F0D003B5FFF738
:10524000B9FF0EBC4243891A1847C046002941D015
:1052500010B4041C4C40A44601230022002900D5B0
:105260004942002800D5404288422CD3012424071B
:10527000A14204D2814202D209011B01F8E7E400F5
:10528000A14204D2814202D249005B00F8E7884281
:1052900001D3401A1A434C08A04202D3001B5C08F9
:1052A00022438C08A04202D3001B9C082243CC0856
:1052B000A04202D3001BDC082243002803D01B09B4
:1052C00001D00909E3E7101C6446002C00D54042D8
:1052D00010BC7047002806D003DB0020C043400804
:1052E00001E08020000607B4024802A140180290A5
:1052F00003BDC046190000000029EBD003B5FFF73D
:10530000A7FF0EBC4243891A1847C0467047C046E3
:1053100042180023002903D0037001309042FBD1D2
:105320007047C04670B5061CB30717D133680F48E5
:105330000F4D1A189A43301C2A420FD104300268CC
:105340000A4BD41894432C4208D104300268074B0E
:10535000D41894432C42F1D000E001300278002AA6
:10536000FBD1FDF773FC301C70BDC046FFFEFEFE96
:10537000808080805B4025303278253032785D0D2A
:105380000A0025732025730D0A00444D31355F4D09
:1053900031420053455249414C20434F4E534F4CEC
:1053A00045007265616479000D0A4279652E2E2EE2
:1053B0000D0A004E4F00203F00257320257320204A
:1053C00025694D485A0056323900202025692E257E
:1053D00030336956002025735254432000444D3425
:1053E00031204F4B00424144204B4559202530325B
:1053F0007800202D2025303278004C43443A253067
:105400003269202D20256900505245535320454EC6
:1054100054455220544F20534156450053495A4554
:105420003A256920555345443A2569204652454559
:105430003A256900535441434B3A002563312048D3
:105440004F5552002D0052544320524541442046AE
:1054500041494C007475726E6564206F6E003C5259
:10546000455345543E0D0A00426164206E756D62DD
:1054700065722E0D0A004241543A2025696D560D81
:105480000A000D0A253032782020005761697469BE
:105490006E6720666F7220646174612E2E2E0D0A75
:1054A00000426164206D6F64656C0D0A0052656195
:1054B000642025730D0A004641494C4544006F663F
:1054C00066004C43442064656275672025730D0AAD
:1054D000004B4244206F75747075742025730D0A5B
:1054E00000436F6E736F6C652074696D656F7574C2
:1054F0002073657420746F202569206D696E757442
:1055000065730D0A00000000005C000C000C7C2894
:105510007C7C447C241048285408000C003844004B
:10552000443800201008103810804000101010007F
:105530004000201008384438007C0064544844542B
:10554000281C107C4C542438542004740C285428F3
:10555000085438005000805000102844282828445F
:105560002810045408384C5C7814787C542838444B
:10557000447C44387C54447C14043844347C107C8F
:10558000007C0020403C7C106C7C40407C087C7C93
:10559000047C7C447C7C14083844787C146848542F
:1055A00024047C047C407C3C403C7C207C6C106C63
:1055B0001C601C64544C7C4400081020447C00088F
:1055C00004088080800408007844780007080400FC
:1055D000000000BF01BF0109050000070007000728
:1055E0000007130A00002000E400FC003F00E70071
:1055F000FC003F002700040F0800000C011E01FF03
:1056000003FF032201E201C2190D00000E001F007A
:1056100011019101FF007E00FC00FE011301110148
:10562000F001E0140A0000EE00FF0111011101BFBA
:1056300001EE00E00130011001050300000F000F32
:105640000A050000F800FE03070701040B0600002E
:10565000000001040707FE03F80F08000000000A1D
:10566000000E001F001F000E000A110900001000AC
:1056700010001000FE00FE001000100010080400D2
:10568000000004800780030D0700001000100010C8
:1056900000100010001008040000000080018001CC
:1056A0000D07000C000FC003F0003C000F00030FBB
:1056B000080000FE00FF01010101010101FF01FEE0
:1056C00010080000000002010201FF01FF010001BB
:1056D0000001100800008601C701610121013101AC
:1056E0001F010E010F08000082008301110111014A
:1056F0001101FF01EE11090000300038002C0026D6
:1057000000FF01FF012000200F08000080009F0122
:105710001F0111011101F101E10F080000FC00FE61
:10572000010B0109010901F901F00F080000010056
:105730000100C101F1013D000F00030F080000EE60
:1057400000FF01110111011101FF01EE0F0800001E
:105750001E003F0121012101A101FF007E0804007C
:105760000000008C018C010804000000048C078CF0
:105770000312090000200070005000D80088008C3F
:1057800001040104011109000048004800480048D4
:1057900000480048004800481109000004010401C5
:1057A0008C018800D80050007000200D0700000216
:1057B000000300B101B9010F0006190D0000F80047
:1057C000FC010603FB06FD0505050505FD05FF05B6
:1057D0000601FC01F8120900008001F0017C004F75
:1057E000004F007C00F00180010F080000FF01FF66
:1057F00001110111011F01FE01E0110900007C00EF
:10580000FE008301010101010101830182110900F0
:1058100000FF01FF010101010101018301FE007C84
:1058200010080000FF01FF01110111011101110118
:1058300011010F080000FF01FF011100110011000C
:10584000110001120900007C00FE0083010101210A
:10585000012101E301E20112090000FF01FF011033
:1058600000100010001000FF01FF010A05000001F8
:1058700001FF01FF0101010B06000100010101010F
:1058800001FF01FF10080000FF01FF0138006C005C
:10589000C6008301010110080000FF01FF010001A3
:1058A0000001000100010001160B0000FF01FF01D3
:1058B0000F003C00F000F0003C000F00FF01FF0172
:1058C00012090000FF01FF010F001C007000E00141
:1058D000FF01FF01130A00007C00FE0083010101AB
:1058E000010101018301FE007C0F080000FF01FFA0
:1058F000012100210021003F001E140A00007C004D
:10590000FE0083010101010101038307FE047C0401
:1059100012090000FF01FF01210021007100DF00DA
:105920008E010001110900008E009F01110111017B
:1059300011011101F301E211090000010001000150
:1059400000FF01FF010100010001110900007F00BB
:10595000FF008001000100018001FF007F110900AC
:105960000007001F007800E001E00178001F000739
:10597000190D00000F007F00F001E0017C001F0006
:105980001F007C00E001F0017F000F12090000837E
:1059900001C7016C00380038006C00C70183011199
:1059A000090000010007001E00F801F8011E0007B1
:1059B0000001120900008101C101610131011901D9
:1059C0000D01070103010004040200007F01090525
:1059D0000000070000000000070B064400FF014420
:1059E000004400FF01440B0600008C001201FF037D
:1059F0002201C40D078200450025009200480144A1
:105A000001820C060000E60019012601C0002001F9
:105A1000070400000000010002080400000000FE6E
:105A20000101020804000000000102FE010B060053
:105A3000008800500020005000880B060000200065
:105A40002000F80020002006030000000400020BE4
:105A50000600002000200020002000200603000097
:105A60000000000109050000800160001800060B1D
:105A7000060000FE00010101010101FE0804000012
:105A800002000200FF010C06000082014101210119
:105A900011010E010B06000082000101110111012C
:105AA000EE0B060000600058004600FF01400B06A8
:105AB00000009F00090109010901F10B060000FE29
:105AC00000110111011101E20B0600000100C101EA
:105AD00031000D00030B060000EE00110111011151
:105AE00001EE0B0600008E00110111011101FE08EC
:105AF00004000000008C018C01080400000000007C
:105B00000208010A05000020005000880004010B73
:105B100006000050005000500050005009050000E1
:105B2000040188005000200B060000020001006103
:105B30000111000E0D077800860132014902390279
:105B400042027C0E07800170004C0043004C007044
:105B50000080010B060000FF01110111011101EE8F
:105B60000B06FE000101010101010101820B06FF8C
:105B70000101010101010182007C0C060000FF010E
:105B800011011101110101010B060000FF011100BB
:105B900011001100010C06FE00010101011101912B
:105BA00000F2010C06FF011000100010001000FFB1
:105BB000010804000000000000FF010704C000000D
:105BC000010001FF0E070000FF0118002400420041
:105BD000810000010C060000FF010001000100012E
:105BE00000010E07FF010C003000C00030000C0067
:105BF000FF010C06FF01060018002000C000FF0195
:105C00000B06FE000101010101010101FE0B06FF6F
:105C10000111001100110011000E0C06FE0001011F
:105C2000010141018101FE020C06FF01110011007A
:105C300011002900C6010B0600008E0011011101A0
:105C40001101E20B06000001000100FF010100014B
:105C50000B06FF000001000100010001FF0D07031A
:105C6000001C006000800160001C00030D071F0085
:105C7000600080017C00800160001F0E07830144EA
:105C800000280010002800440083010D07030004D1
:105C9000000800F00108000400030E078101410123
:105CA0002101110109010501030100000307206121
:105CB000055500000D0C205AC65900000D0C205A45
:105CC000CB55000000070008000A0100181110134E
:105CD0003831303378717073C8C1C0C38881808314
:105CE00084848782C5C4C7C27574777235343732ED
:105CF0001514171202070208020100030109030428
:105D000002040205030500062024282C383C4044E8
:105D1000484C4669726D776172652025735F563213
:105D2000390D0A00252D3130732025732573000DA0
:105D30000A5479706520273C636F6D6D616E643E17
:105D4000203F2720666F7220706172616D730D0AAB
:105D500000557074696D65202575730D0A002573F3
:105D60000D0A0D0A00564F5941474552203E3E202C
:105D70000025630048656C70004E6F207061726191
:105D80006D73004B6579207072657373003C6B65B1
:105D900079313E203C6B6579323E202E2E2E004418
:105DA000756D70206D656D6F7279004C6F61642048
:105DB0006D656D6F727900637400436F6E736F6C05
:105DC000652074696D656F7574003C6D696E7574DE
:105DD00065733E004765742074696D6500747300D7
:105DE0005365742074696D65003C595959594D4D7E
:105DF00044443E203C48484D4D53533E007464009B
:105E00005570646174652074696D65003C6F6666E9
:105E10007365745F696E5F6D696E757465733E005E
:105E20006B6200546F67676C65206B6579626F61A8
:105E30007264206F757470757420746F20636F6E58
:105E4000736F6C6500546F67676C6520646973706D
:105E50006C6179206F757470757420746F20636F36
:105E60006E736F6C65005265616420626174746565
:105E7000727920766F6C746167650000B75300001B
:105E800000000000C51C0000745D0000795D00008A
:105E9000775D0000FF00000069110000835D0000D5
:105EA0008D5D00000D600000000000008D0F0000FF
:105EB0009F5D0000795D00009B5F00000000000016
:105EC0002D100000AB5D0000795D0000B75D0000A3
:105ED0000100000019120000BA5D0000CA5D000058
:105EE000B85D000000000000B50E0000D45D0000A9
:105EF000795D0000DD5D000002000000150F00006C
:105F0000E05D0000E95D0000FD5D000001000000B3
:105F1000550F0000005E00000C5E0000205E0000D7
:105F200000000000ED110000235E0000795D00001C
:105F3000FE5D000000000000C1110000455E000091
:105F4000795D0000215E000000000000A10E00004D
:105F5000665E0000795D0000008001500080025004
:105F600000800350FC3F0150FC3F0250FC3F0350B7
:105F70002578000D0A413A2000202025633A2000B0
:105F80000D0A533A20000D0A4D3A20002020473ACE
:105F900020253032780D0A006661696C00253034A6
:105FA000692D253032692D2530326920253032693E
:105FB0003A253032693A2530326920257300253080
:105FC00032783A253032783A253032692E2530320F
:105FD000690025303278203A202569202569203A49
:105FE0002025303278004E4F205254430025303265
:105FF000783A253032783A253032780025303478B6
:106000002D253032782D2530327820202573000060
:106010003060000034600000386000003C60000028
:10602000406000004460000048600000645D0000C3
:106030004D4F4E00545545005745440054485500B7
:10604000465249005341540053554E00CCC5ED2DE6
:106050001207EE76A609CFA6C6FC205FFD8D1416AA
:10606000A5B8757A3E3979BAAC30388E4526943C5D
:1060700071EA4D1DFC6918F8374D202D5431210C63
:106080007B81EFB98C658A36C3DF9BAF1E308AD621
:10609000E807680B0BE035688B58BB367E32A97A6F
:1060A0000BFA57FD0296BF98D0985FEC4861E9BAA9
:1060B000233F67B933A85C1D8A2E7C20E734169EE7
:1060C000180B638521022479A02300408133DC94DE
:1060D0002FFB993C5492B0BE5BC9D31C43B1DDD8B1
:1060E00082327602251407C50DB09AA840A8A51ED5
:1060F0003236A06AEE5A06EA4519C77715D2A53995
:10610000CCA24A7745067CACAC0C31645B1690DCC3
:1061100089E8C860A5CC40E3F9AC69CE6D5B5875E1
:1061200037C847ABC306D05F490DF7D3728C03EE77
:106130006C76DFD400858D59558EDC03D6F46B0D5B
:10614000ECD3879CB706E117A13110ECD4887F1FF0
:1061500010CA9FC23E76045E1638315A0F19498123
:106160002919BDDE16F74461A154A2E5ED29ADA6BB
:106170006BBA4C0BB86D36E573F542257B305B0589
:10618000AE43AA9562856B34907EA481B93B436689
:1061900044837252D0B598FB7C73D92076A23A82A0
:1061A0007F51C2274FDC7FBB3A9ACD3FBD4DDBE725
:1061B00078C921983DCD24CD2698FB0B4161E9A6F5
:1061C0005592AE9DC6A681AAC9E86FCA34249BA287
:1061D00039A3319056AC2FFE5593AB5EAFDBAC7A52
:1061E00001AF54C3482E984820B32DB68D96445124
:1061F0005735D9D91992415389D0C908086AFF4C3B
:10620000B8392A595B084DCBD85EE3F04527E20444
:10621000E16D1CBEF4C273E99F818CF866229A6D11
:106220000C32D98B088E4F8419611A2FC61CFC22A0
:106230005919B13550CADEB8B48E39C5865277695E
:1062400010C45319A4391728409DE89C34CDE74E5B
:10625000FDA3AB571ACDE49B6787A4D6975534F9B5
:10626000F710871B6628B1090B342D9697B2EE0AFA
:1062700076879DEFC602940373943DD9D2F69ABDFA
:1062800050E96EA6D70ABAFCBC8E6E45B0AFC5DD2C
:10629000D8214F448AEF678FD6D734C920A68C6D9A
:1062A000C459CD6C6D5171B1691A45A79C15BB5687
:1062B000A10CF2318E1A0411C7EED93DCA1EEF4D62
:1062C000E5F968A3B5D55CC5C16A188675FA19E801
:1062D00004F09A6287DBB2C6F97A4206551670B4AA
:1062E0008DC9CCE17C1EF952F86C4D4E29CA48206C
:1062F000B8C0DC4D72A4F7ACA54A4DED02DE7E4E6F
:106300009E8727BDC8F7A2658A4FE9ECE338336F53
:106310006BB7B8AC9AA5FD068DE255B7BD0D51CA55
:10632000DBF620490882928C113F4632352BBC1394
:10633000E8B2B557CDD73C090B6F55A3BA423D2BF8
:10634000E47A8C769718A79840096154979F931325
:10635000418D0E5A1D57932772739799AEC133EF33
:106360004604FB402A8991186AF0D8C200D6DAD9CF
:1063700084DCCEACB8379BFFA463D0F2EF862682D4
:10638000331593FA87F931DD495CB55DAA46C9A793
:10639000D3C5A3CAC2735E9E8018CD4C2D6B9ED60A
:1063A000C325B1365C49024F0FF606057FC5E75598
:1063B000C164E8195A8C5C4CA07B10089EF9DF9CE4
:1063C00092F642BBF35F993A44E0EA1942B16A5946
:1063D000FACB0D34687E4D88A93DF8F0BD47D88FC3
:1063E000CF48814A793F42D30B3E4CD3376D49F1B8
:1063F000DCD59909198CF57D6F5688B98AAC22468F
:10640000751DB5B6DD07FC115E295A04A40861B4F8
:1064100092D62117D06B6871719BE3A4D0A5C4E517
:10642000F091CEC357A5A372F926EABE6A72FF8225
:10643000447D6E09FC643D54AC8B607D510721673F
:1064400081A1FDEFEDF97896CA84E72BA8BD6569B7
:1064500000AEA6C08BF25EF5D21A1C5E6B2D87E1F2
:10646000EB4331A0E997E40A55920BC633B8DEE45A
:10647000C2451C86EF3B9B8D38A25BF5A2EDDE5535
:10648000A4EC8A18EBD67D26EB364049A1FAACC5C0
:106490000DC5FC8B9D077F22F38D36ADE521A2A4AF
:1064A000BA100196DE0159258C2314B440BBF34C7D
:1064B000814A997036E81E722E503D3D97C1ED7F9E
:1064C0004BB852B4A196006A8E8BE47803D5E2DC17
:1064D00039170B3E9084B824B2A9F11D3957D4372F
:1064E00015BD754290AD8BD8BE099505E7FAE5B1AB
:1064F000C667D7B191BC1ED46A671C24219FAD6AC0
:10650000689143F3E317B6E4B0630AF6BE016F1671
:10651000FF8EB9BFB3723A54A98E35FD033FBB9EBF
:10652000CA6FA48BC3F343F5A07EA4DCFD2761C131
:106530001C0CE16A7F2CA21A3583B9517A9F471D42
:1065400014855E84E39F79513CE363398D718F61DB
:106550006AEA2251E7A255A199F1EA8986939C2B18
:1065600052DC0E89DCE2862C8749E4B88F223F900A
:106570007DE7EF369B12BE3D57610D255CD43CEEA6
:106580009E28859E6278FDD97E4C5942190E67A5DA
:10659000662A7D309E3C9A0D02DF1A3062CD016F73
:1065A0009EA7F120791BF10C9B7A59DBCAC16B972E
:1065B00006164EC7C61E1E958EEC8987092D343AE5
:1065C0000056B5C6558F2B6456D5933D7586185524
:1065D00030533627CCC5E4CD05822759FF5FC05321
:1065E0001407A7DF57CC327CDE66E203718EE0042D
:1065F0008E78A02F2BDCD8302427DE6822FA86176D
:106600002E26902434CD9ABAF7BE64D7E68B37494C
:10661000A3E2905C798382609D4A1F0CC099460278
:1066200063AE72E10F9472FB1BC17363F6E2D93063
:1066300096439D0E3D180A6727624CC95BB0C26342
:1066400008C0AA8F51E44A4DEC6FF3CA22371E915D
:10665000ADA047E8BDE8EB903DB1B0452B4F021C23
:106660004FFD5C18A8B35EA7BE55D5B98568EA583A
:10667000E8F308BF02B21A6A9E96D4172C3026039C
:10668000DD138AAFD83C0623B90C70ABB1AD1D2D1C
:10669000B8903F38F4B68D4D200E15607FDC813800
:1066A000D2E58A85AFC1A8EF2D0BAC92344346E901
:1066B000718546AF20B3EB0E3AC8332392D1C0F5B3
:1066C0001F4EEE0C54B6FBDBD4FFF4C3755A0629FB
:1066D000156CBBEE593A52F2DB370C7BB332FFE05C
:1066E000EC03A857E58FB6CBBD9377500DEA3EE794
:1066F000FDF697AF4E1394C31B5426E1914FCEEB9A
:1067000043E9997C8E4AC28DD6C2EBCFF311765AFB
:10671000A26BF083EBAAC386858A744DAC32B17646
:106720006C981BEECC1B5E7A31A29D8164A0FF2188
:106730001A43C92E56E2155BD51DF426143E0CB142
:106740008AE207A477861D0D061177E9CB18FC2F86
:10675000E4B58C0B6C676FEB26C2F7662E4F8D820B
:10676000D9E9F16C867A0A64C638590A59BEB8DB91
:106770000702F509273B3C67A67F19130A95F7A581
:10678000B694D07C96186B4674BA8BAD36AB2A980B
:10679000A2FB6F42B1F42D034AECB88727BF95B92D
:1067A0002BE53197A16990C25145CB2F0FF4313BB6
:1067B000EB232E0C58CC507E1A13FAB2514E61D4F2
:1067C0006A417B048FF176BE8F0068128C5FAECE7B
:1067D000046B19D1DE1068718B65A472F36D578458
:1067E000586169DF2787A014E6EDEFCD94AF72A75B
:1067F000FB6CD6E86220B90676DFA9DE3071AFBA4D
:10680000000E82560F9C9476484DAB9CB87BF7A542
:10681000A7758FCC73C5D4E393E02DBB872A37D4FB
:10682000A282768FFF915B5ACEBCF4BEA5B6107BD8
:1068300052FB43B02E8F8EFDF8215A570C0B7F2B45
:10684000AF5227BD64283C5C052209E8F09BA75B9A
:1068500060D08D9BAE855A2AACE3B6C3F3311FBA24
:10686000652457F81EB401416DC326C6F0FE240D01
:10687000EFDA60108B9FB70B989A9DA84FE131F427
:106880005E1BBA37B4E15A8D94A77E6167AD49D0DB
:106890007124513B16F9057530762087EEFAF4DC49
:1068A00065C7315F197245027DA58779DADCFE3C48
:1068B0005AB14080EA4132C816CC97992545BFB2FB
:1068C0002F70B3A4683E5BB591B13DADE7182B3492
:1068D000B446AE5CB6ABC5997195BA5C5762198087
:1068E00081E27CCEBD8C12622B2AC00A40A61AEE31
:1068F00079F06BF69B2F393E17E643894B6233B430
:10690000DFB0DD983DB0A0F60C502238708E9FA706
:10691000251AEE4543E7C36F56BF1548704B6D9E71
:106920000591C82269D6183978095EB7F6AB9C8004
:10693000DDC82E3298079CFBC6DD2DB59B629C1DE1
:10694000B8A6DF9A5A23D8E6D7F8802AF5F67F73DF
:106950000DA93138A0CCD322E7C416215089761373
:106960003010BCFA861B2990FBF0EB4784A67DE033
:1069700096BDF77137C91B9F45F1312410B1050849
:106980003474342535D17CAE6695698A315CEC6906
:1069900081F799E57F93CB24B687B96980A6987F64
:1069A000B8676C8E7CDC9B395C921988ABB8EE368C
:1069B00021B19240CAFC813958F0F9654EDBBCCE5A
:1069C000D225B7B47DC0315051B1C8B5BFE321C0A5
:1069D0002E8304176068A78D363618152BC28BB727
:1069E0009E3B619FBB8B7506281C6635C6A37D66E2
:1069F000B00E3A228B7D57446CDA241A0E569D1441
:106A00008F6B18D303FD168601A0905DD043329A98
:106A10007E0833A506265689D49DE5C82F37E6FDA6
:106A200032A8D980D659687D0FFDB7FFDFBA3B8603
:106A3000316358B8C4CAFB13719BE63B5256E00A57
:106A4000D00EE94D748E454345913410EC348619CF
:106A5000B58563FFB8755CD67577ADDCA60C0721EC
:106A60000767DE6EBEC49368B3275606351822CB7F
:106A7000E4686E4A597BECD0A2D3013591C72FA3AD
:106A800009D47B26D5A9898DE5FD5AA948CAD40D1C
:106A900023A016A9F90AB56B49F6589FCFDA88C426
:106AA0004616C0DFF24B159B84BB90198322CA495E
:106AB0007D6C5030E3A9CCEE2BE772086F299486E9
:106AC0000C1106351281A54813CE270C2281370BF5
:106AD000884F4489702E69A8D116703B2D76A8F98D
:106AE000D44FBB9E841558F89D363B6E68C9627DB5
:106AF000C38A75129411A65A77A3776B6C660CF152
:106B000075113F197A6A262BB6784E36B9413E4345
:106B1000B6CCCDF7B15E5D7AC722D97B58A8A4FD6B
:106B200030B354995619D2683982359F13201E9379
:106B3000D05DAB11D69AFDAC0B69F4AC1E5D7E0D39
:106B400082E59D77BED085CC936EDFD7BE8B367C39
:106B50009F04739EE9875B58A8D8822861D9C10534
:106B60007612129261F785F5FA1911D53165DB4875
:106B7000F9C4A5C8FE76EFE17461220A35ABC5E61B
:106B8000B13DE74EBB1BC0D330247C3E5049ECA541
:106B90001D4387BB97DEB34FD8415ADDD366D5710D
:106BA000BB9D062D750BB76C3C0FE76003BF3BBE6A
:106BB000BD3C1782EE4CE24AD9FB66FE48862CC9E2
:106BC000F8BFF84440F867D795517B7A970596C18E
:106BD000F7E9C1F5B9F3D6F78A9EBB97E8B0A611DD
:106BE000EAD6FDCEC7A9B6960A1E97A9FF5B78D54F
:106BF000056B7F5B5C94800E1A2C6E83AD47DE4480
:106C0000B0B7A723FFBBB1F8FE4DD4741C02F41833
:106C10001364BA0AE18F003010E32F57038D7E9B77
:106C200079A3055C1AE8B600C5EF06E0A073E4445A
:106C3000BBB5EE5E1C58954B033EDD4298756796DA
:106C4000EB2B13C8303B5916CDC9F260E85E8D0DB1
:106C50007C84798804EE306EC923B8C493D8B4B16B
:106C6000AF09611C20CB7FB5B8685E3DC0EC7720D2
:106C700042C4D6C5BC8B5F7114405B6AB9B3D75BA5
:106C80006BC0D021CDD8A55F446EB28E8AEC76F36E
:106C90008B0EDE8B68A8EB608B0B65E7711EE0B690
:106CA0009BCCC274685ED81F628CC85FFD776FD8BA
:106CB00055DC56FD1F6FBB153AF11DA3F057531855
:106CC000C681E10AB9929EF528D1C7FEE37A155A2A
:106CD000B14E259723D1C4C07A542ECDC6380C5856
:106CE000667CD715960FA4BF1C42B60AC59D2EA17F
:106CF0004B1AFB01AAD67D00BAA61F355A0DAF6B01
:106D0000C9CC2332BF95099E77E799A515FE560495
:106D10001D81FFEDE66E3171944AEEBCC0E6DEDC0B
:106D20005405C33A4EC2A88481DC7065779D063C49
:106D3000AC7BE08390CB19B30B626CC51DDFB8143C
:106D4000C1C80C25466601479A39CB4525D15AC999
:106D5000CEB73AE86EDC0AE57B307743F71606F8E3
:106D6000D3E64F4CBCE02E4681B3D7C518E7CF36EB
:106D7000C26F85AE788A6854B77F8B3E4FC96A74FC
:106D800077586F0B6F7E02D050D9871784C163ED9F
:106D9000039DB8804512FF762551A44ED1F32939C1
:106DA000AE1D9BD960039FDCD0960829E08ECB49AD
:106DB0004AF1EEE94323E7322DEBB56C243771F746
:106DC000885662E83FAC8EFB096254753F4EA91CA1
:106DD0009F84DD43A586CDE9A9E0E1E64A000BCC1E
:106DE00054E33EFEC8D159978143A9C9674AE46775
:106DF000091ECEE9B8D417EE2B36A98038A5A469B0
:106E0000B5D6B2DC0C3667A8A6FC3687513E8ACED2
:106E100082386C1C4129EE5D047B0A020D035AC1C5
:106E200009C300AF6651921D9858C313CA20EEDC07
:106E3000A82A9067B746B74649854A7B3EFB601D46
:106E4000C88D577CBB881610AA441576FAC0065325
:106E5000A245A3B167CE6EBF36D65E46CD3EBA3AE6
:106E6000A92486513D0EF7F9F74767F0ABE5214DB0
:106E700021509942AE88A5B365F970618902562206
:106E800022F63BDEAA7B9279B0C85E2F500B9D792B
:106E90002E0ED8B5307D81FF0267342DE43EBBCF86
:106EA000E344F3FF1BC3339649C43746976D687DAF
:106EB000E1B51DDAA93565CE2717ACBF3C419BACC7
:106EC0009DA9A093BA5F53812B0BC47BF1D1842E73
:106ED000810B101B4869C5051BAC690890E9F8C017
:106EE000FBA81AF76B623CB508E11379D055C1FCD9
:106EF000521FC81C860C7A7632255630629C43A3FA
:106F00003641AE9B8E5F5313970DFC5FBB3E7953AA
:106F1000815D3E5DE8B3B2F1771E14B35F2E659AD2
:106F200029268A7960FFF38E6E1408465354A5888B
:106F300047B6ADE801A8ADACE803B2AF431157AA1C
:106F40004848CC90CED0D6D0FEDA9760D72BDDDE85
:106F500085E9348386622D717512781E21406F8C0D
:106F600035ABA838EE6F78CF9A313E2F3D6327EBD3
:106F7000E3F829D1675C52CEC52F9A1BB60849A900
:106F80004FB37F7CD4EDE72D7A31C0C4D1BB86C925
:106F9000A6752947F5C55CF6923D18B143202F2808
:106FA00029C8E515B1282AA959A58C0B640DAEF5A1
:106FB000DFFC2B069285EB5CB86291A6D0838997A3
:106FC000A1BD1A6BA52890BC86596BAA1EE72B425F
:106FD000DDB32F28B5A6AE626DACC987C9323E3C81
:106FE000B3727C6960EB684DFBD21915DFD965552A
:106FF0007FAFBA0E5D073D05C8433D75DF1FA21385
:107000009D99BB853D6C73EF59969F677E7860F9BB
:10701000CA8FE5016EC25F49A124A775E1F6B1846C
:10702000F6BA49AF822C4901A235C8CAE7CCA10CF7
:107030005B9BE0FA8576A1AB6599B8664AF14FEAA9
:107040005C01B476D8462732779E19AE4DFE616F4B
:10705000DA939A664BC9CF78AC79F88829D4FF4087
:10706000890B7296AAEAB4192130FBCA796C8A8915
:10707000C7EFA8D827DE82CB2EF963599665CFC11A
:10708000D86E724A1835B8D5958F958F749F6383E3
:107090002F6719649739224C2A3E35548BC4E34933
:1070A000B334BC69A10D48B58B0831FD2C2AE658D4
:1070B00096D88E816DE61CAA75EED5E31C04B41635
:1070C000EC027C607945C321D060A3FF576BCD5E95
:1070D000A0B13DC228AF46995D6D43D124946607A7
:1070E000BA67D24FCEA599174219AFD717222D6B89
:1070F000E6D58605DC2966E554BED963E10847BCC0
:10710000CF8B18A9A14FE0E3981D62390AAF22E89E
:1071100002298D181C5A8BA48AF6EE17A966E1AED7
:10712000AC7EA6AA6A723CC9F76950BEF9FA197E0C
:1071300063D0D9FEB0F351BC7ED9F1E3A8A0E862D8
:10714000CD10647377548714FBB4594BD72813744C
:107150002C7B31C85E0978A56025770DA2F0DED4BE
:1071600092D796B963989C76C3903745759231341F
:107170007027D8A29C8BA3F909021B9157F0CEACC3
:1071800001570A53E5429B8501001D0CF1C8B70D5C
:107190004E5866C23D6DDEB1F4AC0680234B1FDE57
:1071A000A8A066B97D87184D8AF5608D29A439415C
:1071B000076D81399A1F5D780A0FEF15EA843C77D5
:1071C00053FF1D0D755737F25C53B0864F7F3D243A
:1071D000AB2F4ED6961011383579F65947A1C0C558
:1071E0008B81B09945F3792E85AA5FE7D7389A331A
:1071F00093E199E92CA908B602117B28861649CBA0
:10720000E98A9F5266C27E6FA997AEB1ADDA70F37C
:10721000BEE2573B8F73FDFA8179695147CEAE7854
:107220002BB25FFF518B24536EA927435C13764723
:107230000784B9B02F1BCEA5885E4D16156A753F21
:107240006EA947D1074DAA7563C41238C71F5F00E6
:10725000E7F5D2A8928A76D8829D469CB15A4940D9
:107260008FAF672A1A19DFB3607C06A173DE654809
:10727000F43559301C40600B2B187CC415DCC583D9
:107280007841B6A4BA26BE871AD986E0D43D3E9886
:10729000684FECCB3B2D1366358024EE98362FC01B
:1072A000BC568DC2DDC6CC96B0CD704BE6A75D86D0
:1072B000B04D171C69132CBE8786AAE082629336F4
:1072C000DD98F7FDEE496CC9818F5EA33A5449F20F
:1072D000655DCB8629A1CC1CB47799AC99D44313B6
:1072E00011B2911A4B092F91C007C96BD4C92E0650
:1072F0000C522DAF9A9A6D12AF00C654B59DB7438C
:1073000031FCC35EEF93BB8E46F2272AD37C111368
:1073100065B345C99282E092FC4009A6C7B2495ABA
:10732000962D6AF1C401619C771B92EB8440391A57
:107330004EF063C41B6C6DE056BBE315C3B8C329A4
:1073400034781BD1F64ED6A10131EC7591C29FABBA
:107350005DEA57DFC60D38855ECC40B2129C5CF406
:10736000EE8758269AC1252B214D9A72D14ABF0C1F
:107370001877E358ECFA6FFDB71D32A34F4128117F
:107380008144038075E538B1D939FDB7C72FEFF2D5
:10739000187D4EEEC48BEC8D5BAE1FF23EBA4902F7
:1073A000A14DE1B4B16A79C329B1F1E24FDC805952
:1073B000A0148AE349713CE52B774EC4F844FE499A
:1073C00075BD3EBF6D6DEBF8EDAB6BC09524FCB7A2
:1073D000EA65C607E58F177490163C5393BD9B0A68
:1073E0004F122CBDC415B1D307B30742D8F4FF998F
:1073F00033A5AC851126263CA9442F16A37F77869A
:1074000003BD60F002EA89424F7DA4A13A5CABCD96
:10741000C110FE37BEC58C90C31F32B30CFA3FBFFC
:10742000FE6241BBE514F1793A38E86841D1A65EC5
:10743000BFCE449DB8AA7D74E2123FA80E07076F25
:107440001E52BDD3A3B0A7DF67F164873DC73FFAE3
:10745000358759ED9D04A7B00FB3B9495B692DF08D
:1074600031D1C80E36BFB606BC028929B47DFD1FD6
:107470004B81D08E1335C8AB66B2E027A6E46569B0
:1074800039A211122777A50FB47068658F28F08E86
:10749000A9C965E59432335DB834168DCE438F604B
:1074A00070C410F6DBEF8EBE15D4C893A6DA077F42
:1074B000E5C1A7BA2F736F636C6721162389AE29C4
:1074C0004291942577CB78B9FFEBD61BA8D2FAB5B9
:1074D000B157C065E58433F2A4110BA7F33569C732
:1074E000AE7FE7144EB40A7D2BFB84A89010A664EF
:1074F000887AB717A0D74CE2940EC6EA46D9B8D717
:1075000080F1340806837512FCB6AA5B7F367DF7DE
:10751000A2F8D0311E0680E4F2128B7FFD9DAD6B88
:10752000FFA3F509CFCA2DD0FFD2DCC6C62DD1737B
:1075300082713BA502890E895FBFED13D54EF80A13
:10754000C0C97F5E3A522DB38648907F04E2A6946C
:10755000779FF42BBD1A4F966A86BC383376EF9B23
:10756000F8660B94A3BFCFC651273DB307C787D793
:1075700060876BECB19D8BAC0E6FDF481EC6A43CE0
:107580000681283C165EC6659D66E3A7B0CD58F11E
:1075900012FE55354DF4A6A6E8691D454D72AB683F
:1075A0002AA79A7C468A6DF906D296E6A7A7672B8A
:1075B000DFB9F6C17083A3C7AED3A75104A834E0E6
:1075C000662AB00155F6CBAA2A374BFBB4040374E4
:1075D0002FD7456105A917369CC58A7AAEEE22C41D
:1075E000422F1A8D5B3DA7E2DC75FDF50DBE05341B
:1075F00039EABC634EC85DDCBC0F9CDA31849782EB
:107600008FE43B1ABB72FC88B9B3FEF2F3254F5AE4
:10761000EFD3BCAEC8084D569FCBA56B553943A8D8
:1076200038EAA0872C34718238CE046BDB26DEDC8E
:10763000161FF28B51693EDA444670C13BB4BA7EE4
:1076400036AE1A98FB1657D3C2EDDE40FDAA541F82
:10765000FE0000013A8B56B79299646B28D458EE1D
:10766000165800812E2AB3BD94857188077E03A029
:10767000026F51E549AC34D6448193E50995C9E3DD
:10768000D008E82BA0E663021BD739B4227842ADBC
:107690002C41C5EBA21C3715015B048A97E788874C
:1076A0001DC78FF921D30BAC24B0446B310F054EAD
:1076B00040A90DD9124035570B4C0B4D16196728B0
:1076C00030C5775E42EF75C810A76AD79E6EDC2F73
:1076D000D95BAA106AB2F706AAF235E2053CE67653
:1076E00024AEB102A87449E59D8DF40ED09F6C764E
:1076F000CF8418DEF869E858170ACB2E2FAF9175A2
:107700002DF92785E8AB7057EB45C93A90F7CFF3D1
:107710005A6A084FCDA7CC0050BC06496263D372A9
:10772000CB76E426D308959C94D824B082913F3C34
:10773000179300F8DA3929C0843D708FC3D12B4FDD
:10774000D4BA1FF477E7E8D148FEF49828A68A6AED
:10775000C27E933D308A0E41334127750E8DBB2783
:1077600009049E1B25A77CA9EB65491BD35B2670EA
:1077700090612B9CCCBA820AFF1BB65B89FAB8EBEE
:107780002457B25D80CAB786E6196395D48687739D
:10779000FDA0B5DDCCF3389E161EC6F0800BFBEFC6
:1077A0000163FF70FB86BD946BD8C55024302AAEB0
:1077B0007D30162945C19D7D1C4BF9C784B8C5B9DC
:1077C00072CF0CC20B94D9160BD131C0C18020CC22
:1077D000E7A69D94A08AC6266B663C6B865FF7720F
:1077E000D859AE6712B6248A46A52DD8E488B89336
:1077F000A183EF7373DD44E8F4CB7F7066C6D6E6F1
:10780000ECD30A4C26DF212DBBF2DE689E8EBCCC69
:107810006F30983B2A0F4CAD8109F55D88333233C8
:1078200057828618445ECBB1FFE54C03CF8BC4333F
:10783000D3502ED8568436B4FE7A8476B57C0DCBE0
:107840000F45870E9FF2158AF5C7FF03F143DD2C24
:10785000417157A06139B507E479834B2E3703395D
:10786000BD17B0F9982D51635DD5D1B11FED01520F
:1078700044C5E3142F156C368622D3D13BDEE79541
:10788000F9C78F1F30264B4818BF10A2EF0E57269E
:10789000E9127C5DFE95B7881A5F5BAA6DA5C801E9
:1078A000B68F2C30D8655F487D3AF3DC4C2AE91B53
:1078B000F22E7F62A7DBAF984CC412D5157D0BA9C1
:1078C000E867636366356D3CDD3366506C73442254
:1078D000A7630FBBD2E8078CB64345F26231C3E51C
:1078E00080EB9E77C71285CEDA5E9B5C7157565E41
:1078F00007DEBDA7DA9B959B5E7C68ACFD9AAD1256
:107900003AD4818B6834465F9236AF4C0EF35508FB
:10791000B5F0FAF47BB87709543CE8EA2A62476F7D
:107920008D3DC26A3D4FD11E951B0F84EAA683117F
:1079300040AE3A11B9FDB49F759566EB04EC223860
:107940009BDFC4FBE15F1D793B3CAE19F4517AE348
:107950009323293057AAE937E9D7EB9BDC45E92D7A
:10796000F47786FF1DD71B3B67BEC7FD51928E463D
:10797000E98064E6B062ED0347B63D19D95DBC62AB
:107980009C0819443BFB558AF838431A374FA164C9
:107990006D2A41FAC11D478A5019FC348F4869AEDF
:1079A0001F55EE24BC1C75FEA43BF318EB8BE5BC05
:1079B000BE7ED43631EA0498C161C9170DFF1E8618
:1079C000E5FB89604B0769B0D0F5B0289F60B8111E
:1079D000447B5742A39CBA515EAE2EC4D35FAB5BCF
:1079E000ED4908DC0CBECF4F9CD436B27AA2660AB1
:1079F0006DF3A28D7B5E28C9B49C962C88D9D95B87
:107A00002F48561DDC1CD4C3C2E6631E93D330A995
:107A1000121AC6D1BF84EB2B2CC1F98EACC3401B0C
:107A2000F5736685848D690D4A556BD80BA1D1A479
:107A30009E6A5D2F0DFA765DE6539229751B59F902
:107A40002E99DDB659C23ACF4126A2A3891A85489C
:107A5000957B6EBFF3CE25513B3F3DB3E0A5D3C030
:107A6000A84647B8F3FCD04CCA6F773BDA4D7BFB96
:107A7000D4FE1904B2AF3660018548B012BCAD8D9A
:107A800056E2DF095D839CB859AF0CADBE89FF1C7F
:107A90007B3BAA487BEBD0B3EA025DEA6C04CE02E2
:107AA000EAD8C874FDB60F5EC66A712709F9445159
:107AB000F23A6CF24E2A9EC1AB517C3F62655D7E0C
:107AC0008F5071E0F70C5AEA93AA988610D084F68A
:107AD000C588F2D04F4F5A529A0FE1E0A74ABC171F
:107AE0003665981D0B03EE2301CFFC31BDF24E0D20
:107AF0003A82C6FF67207BF8967E89A127BEDE9377
:107B00004BEC5067D66AFDF3C47A1002E485DBDAE9
:107B10002CB9FFED16D9EAA7CF9DBB700234E13A2C
:107B200073198022F3B166C3E09D98369DB668C58F
:107B30002A4ABACC24E467A1868C9C3CD6FDE6C1D7
:107B4000CB7CFF0AB9552E8E31D5067E1199E34ABA
:107B5000512DEC603938DB493FBBD43FE400DA3EBD
:107B600074B807F95C7E111BD3342776A415DCA109
:107B7000B2DF69FA6B992251462EF3B291707AAC5A
:107B80009C8BB6636F1F720C151A8CFE420F79EE38
:107B90000164276445CC6A1FCC7A7C820D36B68C92
:107BA0009E71D566F39BBE43D98FE4BBD602F9B56F
:107BB00057CC449C6A640E5483837D0F89801F795F
:107BC0005B46B23F11F5E992DC10A5EC96DC0210A1
:107BD000C5FE853AC184699D8E8E79596912D93B5B
:107BE00015A89B40DDC7DD358BE2A157343D8E766D
:107BF0008CFB7A6A95E2E4C193164088828EA6B522
:107C0000B89EEBD2E39B1C0B9F53B29ED3DC7EB19C
:107C1000650BE6261A32816EA8CE2B3C947477A4AD
:107C2000C8E1866D56CC985648EE33A1C76B1F1637
:107C3000E0D133D891906E22FB5BBB960D6E29A8E4
:107C4000C08806BB9207F53DD533B77A93F774C663
:107C5000911E5CB14896304643955B4B7204EA9A9C
:107C6000E85549EDE01682A841CD2A98CC03A80E2C
:107C70005947389B11ED8D94016F882C5729788FC7
:107C800084F5C5BFC6D8B6F6835B7402659B010B4D
:107C9000FC6BD38FAAF81787EAF54370C723E68CED
:107CA000EFD0D03F0D8A12AB6108D85DDC04616D66
:107CB000FC0C927063690D04E160C7C966DA764016
:107CC0005FD0B76AC9720F2839FFE76B32A9938476
:107CD000FA758FE3B688A3DC026522DF9CD2CC72F2
:107CE0007EE8831677C8809BE214B97F1CD9AC7FED
:107CF000152CF185F05CB403B989A52C393A595398
:107D00000B15C67426370E9A17A3DBB5AB07429640
:107D10002A16A8D731C72760183C37700B8CF79FFD
:107D2000F6CBF35E8F70F74E8F815CBB973FCB171E
:107D30004A1DC133EBE19B7AED4E15691FB6B19434
:107D40003148CC8EAB295112946B03CB1AFD61F5EF
:107D500092325D30CC84666D680557D378F393E535
:107D6000A67FBAED1517F1A4B83ADCBDB5D7025617
:107D700018A68046404DDD7B8B482C82588B7D6851
:107D80003588F9F50944D97127EDDEF1CA2E4D2A5F
:107D9000D706EC9461AAD967061D1212FC8EA5E4E1
:107DA0002AAEB1E021CD950FCF214FF4F98277F3C0
:107DB0002466C1156D207111FC2BE129CE02389388
:107DC00043A301406E6174317869F8066390A7742B
:107DD000B114E2149B9DDC9ABC3F916A4C560E662E
:107DE000B0EEAE991F7BC132275AEF01A96F46361C
:107DF000B9BB47D27396430B82722CC1D83DAF807A
:107E00009743A08CB5EDAA3643DD86F8C39A0B667E
:107E1000911F86E090A52E2D18198C270FE6E24FB2
:107E20000755F94E238FFEF22ADA110AD86680C967
:107E3000B75875973B0E112EB21577B40E2C2C0047
:107E400000A266445BC0593DF605A88766406055B0
:107E5000121ABAD80DE79862865E382280444951DA
:107E6000DB76BA4B3024141B7A78000F7CF97F1E26
:107E7000B9942ADEDC7DDA4829566F597A82274B7D
:107E8000811775A5D0C1CDA786DCE9811B644F4D54
:107E90000A4C21A35042EEBAEE48914D44F0A8118D
:107EA0007F79D9ECA5374E02BA8A208EE81BDE72A4
:107EB000AEB5E42B8ABA439523738914F32BB781AB
:107EC00058764038375A4E5F274530A12A8EFF40FA
:107ED000C5B603A7A98DAAD19C955CAB89DA527C63
:107EE0005327D7646843479D611280FFE0A8E38C65
:107EF000D62863DFBCE8A2EDBEA2439F1AE0945DE2
:107F00004BDC1A11AECF2EBDBA8CBE023EC2BC1FD6
:107F10000E3033E8398F3D6CE6B9A7194DC3A6EF93
:107F2000985D65559734784D7CA4E62625BC7A0487
:107F30000DF965A5CA292566161258DA51ECE8E351
:107F4000BA03A3BB7DA41C44185CE7060E9A62EC3E
:107F5000507B6F087C3FC9FA7B0EF5A4BB6563C1FB
:107F6000BBEE2DAEBEF9188EADA293C5FD9E741565
:107F7000169FA2742B03046B69DFC87D5FADB13E11
:107F8000EDB4EA5E6C0C15903A037056623A4754B1
:107F900016424A8A2FAD98BF52FA0130952B82952E
:107FA000C7F2AF77AB12AB3BF4FD559181FC272AAA
:107FB0008FF40174B0B1ABD041D0F17289B4E78DC8
:107FC0002B52B76DA74899345CE5512A4BD450C762
:107FD0007481658160D8F5806AC45C03D9FDBED622
:107FE000B2F3CA4708A757010494869C76C388D386
:107FF0007A4E08CB6672B8C7B43D4E3062E4DE2FCD
:10800000FFCEF5412E0BCFD8B64908CF649267D684
:10801000F562D6AA87A14A0A921E89E76B3929CE52
:108020006F350334BCA69E14ED8794BF348EB8C858
:10803000D4491B5DD92D4E36E6A8EA52E8043884AF
:10804000EE9AAD1AD49CBBF40AA00ED56C2F0ED8B4
:10805000AF47E1F903FD3C1F67782F5BA8527634E8
:108060005A73A7276EAB48BD34FDE6ED545CAF05EF
:1080700032800873B24D71DCD9267C8A058A6EAFD6
:10808000B7FF06ED0C2CB8AE1E92E5CA5F65941ED4
:108090007FFBFFF9032F993C243AC74CDBB9BF0D96
:1080A000A36040F9FDB120BE3D295BC2362837A848
:1080B00059376098C0E848F86807B6B07552D83AA2
:1080C0007F8744243A64A0CE7E52A9DCF5862A221A
:1080D000F8FB3E95CE12F6338A57C485720A6A5170
:1080E000FF73E1955D6C25745999F16BF005785338
:1080F0003ED39B9E172F8098AD78DDA2DC65375567
:10810000AA0E582271E4242CACA84465679A7CAD71
:10811000F170A95D3F303953F9A844625848656849
:10812000AD97A0BAE47003EC636CE8D7CF0F039669
:10813000956408A4923FEC2D4A908E7063E02ACC9F
:10814000C61C4A5623412CC8C0DC9B772037C6A8E2
:10815000291B358C866A4F4CEF05F3B92103F4DBFC
:108160006BF5B958BC91E62EAE26A84367EC0D65B9
:10817000B6903E50AFFD8AD99496C077E7F847A3F2
:10818000E8FC3620B9BCE9E8E7021F98AB56623D2F
:1081900058FDB1B6C8763B42CE3555E7F0116EF8C2
:1081A00046713187825C25365D5BFA939A8AAA26EE
:1081B000AAA0622201131CA4C845B2AD7EE1DB4433
:1081C000F1B64A55C395FABEF1B60F686541604FE6
:1081D000A5D4DA91FE8BCF043CEBC44DAA1BA89F1B
:1081E000705304C7D0239ECD11F1324DD2BBD9DDDF
:1081F00035D84A2D46E450B3D84DD1006865DFDF4D
:108200005AB0F4E9435C5BD517E0B3BED1BAE5746C
:108210002D669BC787BF4BEEE31E3AF5F864D82165
:1082200095AFD537A7385B012BDCD9985F29AA8C8D
:10823000376C0AD73F6FF2430B2CCBFCBB34DAE12F
:10824000C7CFAC45176836ED44EFDDF4A9E68645A7
:10825000E2200A3E6C3BBA7195BE3FD3BED4F3C454
:10826000B624D966C2555A9CCEBBD4740EB1A5AC07
:10827000A9ACE506701033C30541E8FD703AC0FAB9
:108280007F6F6036E9D1F41860F4C198FD81CCFCB1
:108290002AB14C15FA5219C904B648AA988CE1794A
:1082A00015882235CA2F4DD19605FBA8EBA461D6BF
:1082B000803ED1A73D44ED49B0AB1F599915B6D7C3
:1082C0005626AEDFBE049A19ACBDCE25CBDFB65A1A
:1082D0002EBD102ED4DF109757FA75CAEC3DD6DCB0
:1082E000D490A2F377867359A26618A49ACBB5B935
:1082F000FC6B19A134C619AABD400A6C13D39BB6F6
:108300006BD5E7D471797D501669062BE129842855
:108310006585A6DF9510D3F9CC3429DD3854A62D18
:108320006A4036CB4ECFA7741BED5DC46541FF8A12
:10833000EDC3FCBF4D66C459BAE5E5AF494E9ECBCF
:1083400044616D67ADD991A4B1A3910AA86E431D94
:10835000B9613F1BFB5786D116AD8A850686F83B6F
:108360002DB39742E975E93FC4EAD17B76B77050E7
:108370006EDAE9B4EAC4DC8ADCD3AA7FCDBC5387C9
:1083800012CD28F7D3A89C9C5119D3A01A0D2AA36B
:10839000EEC7F75FD2AAD71C38BAAF24511B0842E8
:1083A000E3C970195D25EC70A49EEB1E7A412B4742
:1083B0007AA2AE75E6688ACEE86DE2BD11A44D9F43
:1083C000C49AEA75C9F8243ACAD40E3B2E26D3863D
:1083D00072520A5ED8AF9115B01A006AAE5C229A4A
:1083E00081BD2D98495445D5B6C7E8EE8A4E243252
:1083F00015ED6E7836096109052047D8879E1F263E
:1084000097389D8F3A9D7494A23D79C4D2550F2C14
:1084100014563515F3D804CDFEC6914C26A4139EF0
:108420001FE1D39C1DFE392FDE2B0A714527AD9825
:108430009BF0AD38CF63B9969ADF98997DCB7E5F7C
:10844000A459026181248A6329C3CDF3E7CFFE6971
:108450006DBD4BEE4DA134AE6A36D0283904F9E536
:108460001BF65D9066450D170A360A5932A1955CD8
:10847000171F385997A61E02829ADAC6F0CE7326C5
:108480007085DA588A247E7DD34A7EF20DECD97647
:108490002405A53F84AE39416A0FE9A796D4C929BE
:1084A0004EEEBE659C36A927C5203E8CE9718544F9
:1084B000543977DF3943AFA88AA4EA1E80FF28F138
:1084C0009352988B9138DDC44359C315513CA9C3CD
:1084D0004420A9336BB1DBF15499F701E2C9D422EE
:1084E0004E89D1DC5DCA5ED2843AB4B8DD7B3BFEF6
:1084F00094F32A35269A390ED72A030665931480F9
:108500009D0C53D8DD24F7B7CDAE632150DD8C1F11
:10851000D2FFF28F32F24637314C105BF980F5A76B
:10852000B3539EAD5AAC68F3BF64251A53A00376CB
:10853000697ACA53ACD263FB7B21F4CE5DE886A591
:108540007C9E78ACF90BAD05BD9745DA999361F542
:10855000091927CE39F9F4ABA9E1351D864833B2A4
:1085600098A1EB227843AB165D2691150DD5B97015
:108570009187C0AA58D86BC55819601A0CAB07B9B7
:1085800037FD0EC5E185F7D4581B6F7F4E858D747E
:10859000211F442871921561A166A4BD72D01DB33C
:1085A0009D4B9AA47624916613F35F4C0126DFC895
:1085B0000DABD2D4F844611DD363A9E4AF0B47B22D
:1085C0009FFC7683771FFE6D141661ABCBDDBFA1D8
:1085D000C6E376DAF5CA556BBA3D427B1261558C1B
:1085E000B1B74D0B798EE7555CB7D50F52E6B2B5F2
:1085F0001FB4F3AE768317970FD1F1BEF81B5A372D
:1086000047F31C745059BD95A06671E6C75599BED5
:1086100071E3579116E789E6FF91E751EDEA2EC421
:108620007377BB30C6EC66AC1EB91E57FD20FA2925
:10863000E4457B9F0912198C66E5C19FC1CA65712B
:1086400004ABA2E17B31644C370C14AF60739042F1
:10865000A99934DEA89117C585D09F16242FE19AD9
:1086600021E6C569A2228F486B763705C949D1A397
:10867000A1B9B1D024ADDF950C3CB297B42A7ED11C
:108680009D59653EA55C53D355ADD56B58115FBC64
:10869000888216F3D3980669C026960E7D9DC0E7A2
:1086A000BD73D1664A3BFB6F2A90C5C488BF079152
:1086B000C546B0AE1269CCE02498CEE3FB6EA08133
:1086C00027CF3A936D759AE5038C92F6370F878B17
:1086D0008995AE76C1431634B3A59784F027603DE3
:1086E00011593AD116CD7A3D78F940879EA15EB8EE
:1086F000B651852685EDC37CD99EF56040DF9EEF9F
:108700008ECA5161EA5A2E765EDC427715A044E4A7
:1087100044546A065C7B2400F8E1E2C9C38D00730F
:10872000F7F4E761D265E3482E284026F2D17C4178
:10873000540F0A0CD895B4FBABFC39FBF0D810AA47
:108740009377EC389EC73D4191A2C0A27BF902A568
:10875000FC487706D62221AF9362AAB9BF31F6B999
:10876000B958BF2EBFBD30AE6B8EB99010BBED03B4
:108770002227DEA5497C2081769F0CA030F7F7D315
:10878000F50FDA26B57EB197DC094611736FB7CDC8
:1087900090AFE1A8128682A39931CF4BA07718B58C
:1087A000D5F0CED825CCB7CE4F6F2DCF626A64718D
:1087B0006269870BDAEE6E070683AB1DAE67E9537D
:1087C0000C342286E98A14EE2355204BB9EC79A8A3
:1087D000130947F9150E78EBE4765D33A240C5ED39
:1087E000A22A0E90AC6247610F0ED97AEE21EEDF1D
:1087F0006671F6515659119D73707454A4FE5770EA
:108800007A31C860FAEB4BD9D31414C5DFA0514CB0
:10881000EFB0A520DFD8F0006863D843EA0214D196
:1088200034F295FC911B76CD341453B55923F624BC
:10883000B245B5DA21B9E287A68DFD8C3FF8BCA020
:1088400038886B1386B923AD667BB258B16E7E75DE
:108850003550E1E6F3200B43E8D0CCD48DCA6FE06D
:10886000D0F34B12522ED011F16F4543152DD31872
:108870008314DF95809916649D1164EEAB10FC148F
:1088800050BB4E89CFAAE5077E5717C5C5CFBEC0DE
:108890008AC1D5E446295FCC4DB1AF63DB488CFA81
:1088A000A68C4BE30116109E9B122FD471894EB1FA
:1088B000B2FFB2C103AD9E03F7830A49C7E49A7EB3
:1088C000C258EC91415F4250DBCB40E81B808B7675
:1088D0000BEBB17E3DFBE4080EE422FD37BF6AB12D
:1088E000419D71BC14C419CEAE42FE27AA21B9EE37
:1088F000D3973B7291D3E352E746C44A73AEDCD6BA
:10890000689927A992AD59828DE8981E9B9345B529
:10891000B61420BA833D5F28FC02086EDBB219B89A
:108920007368ABB5FC5D4103C5005CC4B6A3E67FCC
:1089300032859A59E6AEB95E96B7104701A5E00EAA
:10894000A80533B8DC033B136C73935338F2D8A6F5
:10895000B64AF1C906AD8EE9E0178E22C7A78B692A
:108960008C6C9989D8674D35B2852FEA4CABE73EC0
:10897000E48351DA5283CEE2AE205B70E6A8FD08B4
:10898000F18B1E39666B738E75C1A5B805A3C8122D
:10899000C8CFD47231C09A122FB0FEF18B05CC0033
:1089A000E918B98735D15E060B57D2182C1A30E575
:1089B000FB83D644A8ACFDAF91AE8F8EFA1A161B7E
:1089C000768FA340B22F981ECA8B8857C7AB8CB83E
:1089D000587148C895880BDAF62CC263E333769D4C
:1089E0009DF00F20647415BEEEDF60171F6AA35A56
:1089F000F7AECC60DDA4835F68BA1838AC27BA96AE
:108A0000BC28785A99FF89BF352972498D9CC4FCCE
:108A100041874C4E66C0F21DEBFCDD95D6213A0E27
:108A2000874E1FFA20C69CE3D13AAABA52F83907FA
:108A30003F8F9F120DCE52E1D975546C77669686A2
:108A4000FECF22A0A57ABAAD22402D0F9CA6070129
:108A5000A9B6A19A8B523EA0DD9A3005DF991CB9C8
:108A6000DA7E26CEB9E4A1B8BF90F2001ACFBC03DB
:108A70007532CEE167052C6527D0E10374023CE72F
:108A8000DBA4A7D8DEA708C56801A53E5347982BED
:108A9000B0A6694784D694FB418EA7073A0E5A6A5E
:108AA000FDCD14F6C1E2141B2815E71DA10E5CCD07
:108AB000D9D4E8AC6C5C431409A159CF61177FD4B9
:108AC0005F818AAF1B45C4F5EFA51CCDE1A1AB5971
:108AD000B742A01F7B692328636BFBA8F5A05A5EF1
:108AE000397EAA8B97364DD2B6BDE0DBAA49921FDC
:108AF000FAB0D238DAF116F32A84550B07F341F9AC
:108B00001B8D3C4CDD840A3B7A7E0B7AF8007E8616
:108B100019CA37236A31A803E2CCA69951F10A4356
:108B200054FB30D3F5F1C9A7AF412293954E2F994D
:108B3000E02E2D13F03526459014A5326C10A2348A
:108B40006E2ADE85D859DD9D2B4CD8EF21DE686575
:108B50002E77B21C564C50BF6788B783462ABD1D7E
:108B600042BB21A16F918E4411E648B147CBDB3661
:108B70000FB9F0C3A6F9B0A4FC2FFCE018472B35C1
:108B8000AF8BFC8F8C4102CF55F25DBE1659D84495
:108B9000F9158E4D570947A1D28D2DD5ACF9C89C3A
:108BA0009183B6FAB95F5A3EEE4D7801027E788025
:108BB000C0DB092CFE4C1B677350B6BA5C0F71E02A
:108BC0004D36FA026B1293D0E1A73939DAB4A050CE
:108BD000C1CA160BCEFD308B3714DB0B618D63776A
:108BE000669EF58F7D9B75B2A080FB8F374358251D
:108BF000C9F877D0EFBB7543DA1E1E199E9BD2F0E1
:108C000051EF04D5C76C4DADD14833866C52FC4052
:108C1000DA19B655DA948F0FC06336FA7E087B2EC8
:108C20000D55912EAA0775F4B5F3D24A08E9A41F91
:108C30001C2F29D2E50EC5F0662596AC2E13F274D2
:108C40008104E986B65269068584E5FBC73B540278
:108C50001EF957273121F8D867B6189EC43AA1F8F3
:108C600048C23DE6F0AC946BC90FE31FA30F862604
:108C7000B8DEC85A64724E281E4821B44CC7780921
:108C8000EBA5F80281B17C94D6B15CC13C4934FFBC
:108C900098F3F84BDC0146B66398AFD02AB629E8C2
:108CA000D0633590026E5BADB0E2DE7536FB6C7F53
:108CB00094B601A7DF06E9EC4D2AC9D166D4DEDE01
:108CC0006A98351D1C771241ECED67ADC53B6BC052
:108CD00025DD25D8B53D154848A5296C98C043FF2A
:108CE000D3A03478FF4B8B9543F995F7E14DF6BF50
:108CF000DBBE2D625300D2F4C5D4DADEC2F8DA95B9
:108D00009E09588FB3FC322410E2DD9B2560602F52
:108D100062E4737B0083E7298983A0C3C9D8EAE0B2
:108D2000959F81CB78A23F4FE1C18407ADFE03C37D
:108D3000FBAB3A4DB13E8422F07260325A3D53672C
:108D400072D921AF745616ADDB38FFAA5D1CFB9DAE
:108D5000F21D84A36C5E24F56323F43EBBFA61E547
:108D60000038ED8A2998F426EF3233E0148698977C
:108D70002E9BE87EFB017E431A5B4021EC5878A1D4
:108D800042729A2EBF412D9827617B135BC85BEA24
:108D9000DCF450BDBEE3D585011EB7D8A1FB5F2032
:108DA0001C27C18BC4B72E78636862FE8FD2F35341
:108DB000E2532769D56BEC4E6F7CD52F277F844D0E
:108DC0004727CDB3677B7E6EF8AAE7A5B0D70F53D0
:108DD000DB00DB1773F9E5678E93EAAC05AC4B0259
:108DE000783541CEBA4A4B58009DF89111AC527873
:108DF00020068A29F62CA18864FCA837481EBCEA04
:108E0000EAA8F640A799393564DB9C240248E94C6E
:108E10006F40CB1EEB979F381983FBBAA80AAC1E94
:108E200045A14EDB1021651F78A716B6D521443A1F
:108E300051D46BB88552A17A61FFD439C883AEFB97
:108E40009AE6CFC7E45A68D43C6443765509BCB36C
:108E500050168FB6325C65093F4D925B534F943983
:108E6000FE4AA4AAD1447C022DC0B7BCD9292365EF
:108E7000C54821D39F5810F49AC3ECF57E6CA180AD
:108E80000EAF7F24541CAB2F64EFA13E0D08CE56CD
:108E900028C20AF97539298B4E52AE896BE74A28E8
:108EA000D1CD52FFDC8957904AB89F1ECC3821D5CE
:108EB000BEEA61E94315F2DD1E13AB93DC399DB3C5
:108EC000B7FC06E3EACDAD81EF72D6E183768AB2D4
:108ED000CDC7FE0719124ECCC83A952DEA5AFBAD04
:108EE00098BE96BD22ED5E72563AE2245E2F890549
:108EF000A52160484C22BB89E0B49F8202A956B1EB
:108F0000DD081D44466D6E5F48C6ACA98ADD3FC1D1
:108F100026D57C6AA327F80D4A335D476D2058306B
:108F20003AC5C0CDE0B8A1E1B74BA49CAF07E6E7D6
:108F300057C7047090718E935D77928527293852B8
:108F4000E9A9FD8C9EE7AA8AC77FEFF16653F63444
:108F5000BE0B26386B2CFB39153BCB9565B283F9DC
:108F6000C25B03670CE7FAE559FC2E2F543EA6E4DA
:108F7000E26EEA33A5B5DCB3B53207AC0A1D76184C
:108F8000D131D71BA4AB557C4F0F361169D1DE060A
:108F90006AB7FF392F04E1D736FC026A4E5F62BB25
:108FA00012388E283750DF74724DB17B0DF3E62FE7
:108FB000AC05712C74032CFF7390ABDBA85F68D7F2
:108FC000FEECF66018FF11E190D999B9CAB62040BD
:108FD000750E4AFEC72B8D5F0186E4F55A266B019C
:108FE0002619E26797ECBA98EF0905C91FFE179D8D
:108FF0009C827C117CB844C8080AB6473B77B6917E
:10900000290A4ACDEBF8E3A91A7C4AB79663C84906
:1090100020F65997268C376166EEFDED4A40987030
:10902000F8B1D7DF08AA3D683FECFC8A314967E315
:10903000AF796A7FD86987F6382D4E39E6DB7D96A1
:10904000A2F897414D734A240AB47B50074A42075D
:1090500078AE4029FEFDC091C33D777AC3690D7C8F
:109060007C2A39F0138A2B78DD7E541A0766A5A274
:10907000CD6F030F883653883A16F602DC8B2E8BA1
:109080007D8F57AC875669109FA94BF5AFA20CFB9B
:10909000B094BC45D9132F436F6F1095F297F0A091
:1090A000CCD15D274FD06CB42C4FBDE625DC69C414
:1090B0001079F09A59B2843A389460645ACC4B8152
:1090C0008AE5E88042DCC56A661228055AA52AC7E7
:1090D0002B810B8D1637AFBE6AC43ABAA889E5DE7C
:1090E000DD2082F99E860A3600DFE98881D86AEAA7
:1090F00011BB50844AB61D2045C8EF81026D66C77A
:10910000BB27E2F6C16F7D4E181AB21E87E2E92432
:109110003B5ECD847ACB67CA6D62C2521AB065736A
:109120004B363CBE5D417F984087BB7D1B4BD1B524
:109130003AEB3DA07D1420405239DAFC1548FC3D45
:10914000521250938F91A886A9BC182F10A1601CB1
:109150001C4FD93347BC066C240D486FD30B87B521
:109160005D9BC2C0661783101776795304C720DF52
:10917000ED481F297A3C14E0B1B81464AEF1E23531
:109180007DAEFF36190770194FCEBA175E377A7366
:10919000EF3F9732D0321DEBC78C70ED4E36193D44
:1091A0000F38A40FA46FA296D24983E5B8B241A2AA
:1091B0009BD00B5D2299242523D4A434E43328AB1F
:1091C0003AA4EDD15596082CEB4D814047FB9066B3
:1091D000A53993E47B309A056567DA593B99725655
:1091E000497B75F4EB1681F486DC7ED02ACC4A24C8
:1091F000F5F380023E8CBEF1B92B325EDD02B0EB9E
:109200004EB65503EC5C841121F2262A04DDD86A9F
:109210007D00E206FD73FAA11D5AD8ED5130562D9E
:10922000E34953C1865957021305F6F441BE3A305B
:10923000E90C85398A1D983805048EF3642C196C65
:10924000CA66387288E78E75EABB7C9B166D8651BC
:109250003C7E53BB5A25AB35E353FC846FAAB2D195
:10926000D288E175717B2E4C6C76F8DF940A308DD4
:10927000F3F7CBDD73DA937E2E34DB1F71183E419A
:109280007E602420A8E54B2678CD53AE2DF31E0139
:109290009A594EE04AFE93A259C67EC8C76CB0B830
:1092A0003454907406ECD82A18AAA615CB568274AA
:1092B000B4052F418F6AB6F3974A79E10585319E4F
:1092C000EACD50D006516F8C45AA056860AE77CEC6
:1092D000ED655C6C264217920AA4BC3772E96D4CAE
:1092E0000F34B78209273C72AA85E1A3B7A6219162
:1092F00094BD9930C5CC7D443D6E33D092059B2200
:1093000033502DED55066AE4E7032A109ECCAFF1E9
:1093100016051E21B47C8773EA89AECC8836883264
:10932000F31FED2DD5B76933109C9B70102EF446BA
:10933000447D6438628B18D59C6F3FE269B5B923D0
:1093400088DB4B31DEF2BB9AE0D24A4912E5564E39
:10935000F254795144A3E1C6BA862F7B0B0A7B7481
:109360004BA3019C2E172C0DF19D1E438665FBBD62
:109370008F251F11A3383D42A4195E141802BA3F6D
:1093800014B1DF35F68594D03071375ABECED43360
:10939000D15BEB9ED6C8260B827073C95786C25923
:1093A0000C6B1606F54BB567F452F69E9FBC46B1A2
:1093B000308CC1ACD9E4A32332D29A32FF311AB235
:1093C00047F98F6864FB3FF105BD0C939E6C79AB48
:1093D00072FEC8236BB0A72D517DB78F5C1004813E
:1093E0009CE895A737FB4E2D4FB6B91CDD2166359D
:1093F00070FCF2371D78AF9DDFE73CBFA0239DCD09
:10940000F796457298BF9937B710819CE0F2C36E0A
:10941000ABBE03ABB7D12218FADEA2775B3AFB559D
:10942000A0F6831FFC89AA89939B09669F213CF8BB
:10943000B5F4E4654DF6CA4C5F4A0A7102E42E9217
:109440007D367C8471751E037F7B37CC6E021737A7
:10945000B85A59C37E0004E8D6FB0D7F9C3CDFCB95
:109460006B1B7818FE2122B00067141EE4DB6D0B25
:1094700099173683EA42AE9B555C1A574550871DB3
:1094800020578EB3FB384E80255E2DAC969CF0782D
:10949000BF7E57423126EEBF202AA38702E49A1CE2
:1094A0003231B6BCC6922A13151AB27C82A7D25B9F
:1094B000BAFC2E6D98A4EB9C45B14A70FBBFF33407
:1094C000B8F2BA0AFDC334B41C459F407B95F6B18F
:1094D00011A81A0EBF3F012D857B21A9C7F25E3B63
:1094E000896C1A447E11602816CDBA739C40B1591C
:1094F0006BAC2C96C3EC20FF99D65AAE85EE4BF799
:10950000C51EF5B6C3144A0FA76D44A644FF574BBA
:109510000D132FE9AA76BD8FCC1516596A689CE900
:10952000C5982F09C27A0415FB8A48927C65614769
:10953000E59BD671B849ED6B754AF82A5A4F6937E1
:109540005CEC5C64F13F1DAB9802DE197C97DB5349
:10955000E131D9D79CD3A799CF3357121D951B91D1
:109560001F0653FDDCB01D38CA121ECFC2833975E9
:10957000416D1C6A25B3AA35B3346236371557F2EC
:109580009EC1E089D15BBA46BD3B923FDB2CD0A2A5
:10959000DBF83AC2AE0E10AC8D87CA2F5EE6402CC7
:1095A000C27AB699CE14F0884F2D9668F976D50711
:1095B0003E3B5AC932C840CEEE65A415316AE92255
:1095C00011F1F117BF8021DA9D2CA2E8E26F7E3AFB
:1095D0008ED8F2C3F54B34788A75F28ABB8DA9E038
:1095E000F9C718A80AF8406394AF4810F1808D9C21
:1095F000B121785420C5EB35CB3BC89A1C5FDA26E5
:109600002B127013B24934366C2ACF40A355C136A1
:1096100064404AE856ADC594C265EA9A13AE2E304E
:10962000D5476BFFEA1CA842EE20609CFFEEE2D714
:10963000B04A1C7C8E691F64C9E5C566FDB9DF535D
:10964000F931F2FFB707C15980993B1C4C01307DBD
:10965000101FDC72DDB8D2D6D41B4F5CE17B849541
:109660009B910BF6D11F9FBD9485FF03D4CA9B909D
:1096700014867F314D9197B217560802F84197E84A
:1096800041A933F99A2B2BED1E3AB3B9FB819F8187
:1096900037C519EC9946F5D96D8EE85E9DA9E4129F
:1096A0005751E887A12B07CE518C160932E7C2919A
:1096B000FEA66E44A79EA3C4470ABB501216CE7BDB
:1096C000446E2FDBD87A4D8CEDFF302E7A8E701ED3
:1096D000DDF300D13460E2818AE26B3A6862FCA576
:1096E0002832E2F7285EADC2C9AEED1F5B1DC38A0A
:1096F000B97350AB06C598FB59F8E703E44C904E9C
:109700007908A18085473FB2EA53AE8C1D33A72F5D
:1097100070135DA52232DFFCF4F56CEA794C76A17A
:10972000EC25030F7C6E7134DFA578BF7F50958DDB
:109730006C395CC448158DB958007095F7CE2C383B
:109740005D37F2E9670CB8D31D3B2D824FEE4243E3
:109750006FDFE389C5281D3B3896233BCC3362A2DB
:10976000AF86D35537CEC84093FB1F290CF8F4E7DA
:10977000F0EF38766FE53B2CB7BA47746D1CBC0828
:10978000CAE24622A85FD85AEA0A9F5454DBA8EFDF
:10979000882F2D55FE3723CC5AE5F071EAFC6C93E7
:1097A0009095F6D8AB36CEAE6DEB07B21B559E0842
:1097B00008AE0E71F2B57419B0EE87D3625B7743D1
:1097C000624EBDE65D316C07ACDB2253B3C2F0FEE6
:1097D00068C646D21EDE703E792666D661A9F5A31C
:1097E0003F6340A2233E58A20A8CD680BA056F0D73
:1097F000AE1F8AD4A2B361CA664C24DEBEB50A0588
:1098000003F85E3F67232CC83DE4D06AC314E40824
:10981000EB56CF3907BBAA4DA2B288FB3FAE7D1DE8
:109820003931E5EAA416A5F970609CBAE7646C9535
:109830006DD4C1CB00C81AF5C2EC6527AF7145BA2B
:109840001D62C9AEA212D0D4B3BC840AA37DB78F67
:10985000664853586DF58CFAD2CFC6FD5A501106A2
:109860002048B6145604AE51F4F6B8814D15706711
:1098700016AD0BC3EE9753CB0ADF8325B18EAA42F8
:10988000A94DD7BEF24FC35C3652A795CDF87A07E3
:10989000110A352A03E4B1559F44F80F4F75E13A98
:1098A000840B11E0D8CF058623A0745F56AEC5D1D6
:1098B0003766A484FADBBAE8C6E1B00AB1067FE6EF
:1098C000FE2BC6FABEBA30E11B4CFFC26B9EB35CE6
:1098D000BA58D2D41285E4BBADE4BE1F06B467F912
:1098E000B51BA7953CC142C56605307086D2E7D24C
:1098F000C238F0775A617116E03E1730A22923F280
:10990000318415A4412EE78123ABA4A2F6FDE466C1
:10991000F5686D7CE078606B300068DA7DD7E00F29
:109920001DDA7A6D4A378811A7DA1962C808441817
:10993000DB14D3DAC954F684D6D9AC81CED83891A9
:10994000FC98772D28AC41D10C2A36FB8415914820
:109950006E387EE764E14E51687CF269865BFF1FDA
:109960007141D7757346FA5008326ACCE41C03CAB9
:109970004D1938A3476DF3184103360AF6BAC1E012
:109980006E29AF85F03AEBCD222DB3D7C9E6C2E4FC
:10999000DD438AB0FBF3A64BAAA59496C416426A8F
:1099A0005828F72E4CEA5729495A8FA85042068268
:1099B000F416C2308F0644A8E0C4987F4A888A070C
:1099C000FB24B0BFFA62533A1F18BF1B09E5C1441C
:1099D00000CBB3BA0E63CB7925DAF12ED9E701B506
:1099E000DF3623892DD63ABB3FC2691DB24345609D
:1099F000EB2EBF24FEF546856830547DA9C7490982
:109A0000F1741CA628BA6C897CFFDCDD82CFBBF325
:109A10002F3C0B2A225FE1A6C791CD149B530B5C10
:109A200079CDB1996896E2DC0950F5A4DCAB2287C8
:109A3000B1FFA39C04C7748319D2A30A4C58ECD17C
:109A400097587B84590A0554C8B1C5C2DA52AFCEC3
:109A50003C1D5FCE2AADF3B3016B2E937B3FE77ABB
:109A60009BB8EFDBD41A981C1A477E29BC25C3B9D2
:109A7000FEE196EDC4A8639661B4DDF552B868883E
:109A80007E5A91BB8BBF7DC58F77849CEB1A36FACB
:109A9000A741497989AF904DAE8B8505D2243676A2
:109AA0008491D5EC39BBE9C9D0F7A8BD931D1BA1A2
:109AB0005E0D63D4D1DF3F474CE512CBF72FCDF7D6
:109AC000B9D7255BE41990C0CD82EB40F914ADAD58
:109AD0005C9A6D632BD1724201E5152A7C66D985AB
:109AE0001C2458D8431D7A76F7D129B81FB1F43217
:109AF0004AFF0763ACB489A08730A6312CACD29C56
:109B0000EAB9BAB4CA73A23378F46FCDF5195A978B
:109B10003D762DF7BE79F01B80A7EBA0DEFC94BC50
:109B20005295DCDFFC9275D9FBE60FE1189070F2DC
:109B3000845B729E63761898B656E1C344DA5C95EE
:109B400041B0367BDA57F016459ABB1F877DEF94FC
:109B50000659C637FD2694038211F4E11E0D272213
:109B600049AA1367C8DEFC88A99F5DA64B3E12492F
:109B7000C794DCCFD6492A73503D9BB24947DECF0C
:109B8000528F2F24F376010668AF2454D8B60F6C99
:109B9000E3B7858BD82EAE221998AA0FFCB10B6DB6
:109BA0000A78F414D2C445C4169ADE6F9E6300325C
:109BB0006839BCCEE62605880D6B79F244038D200A
:109BC0001175C5E84AEADC92DAAE0ABD3A5AA11B21
:109BD000832C56FEAA63D33C69EEBEDB217453C6C8
:109BE0006A98AE262F78618DAE3B861BD268F2BD97
:109BF00031A6642F6773B60595E73A766197B87911
:109C0000E1C728CF617A74382BDF5C585AB94AAB68
:109C100013F9386A958BA213E6B178A9E609819009
:109C2000227CB2AE47CFC94DC1A33293983B2FA738
:109C30001C6E1066C989804B4D2CC49EC1B9C548A5
:109C4000853CFE4820D05227FD4A66AA0304050A37
:109C500008060BFF0209070D010C00FF20256920F3
:109C600025692025692D256900202025633A25696D
:109C700000202020205F5F7C002C0061004469737D
:109C800070206F66660D0A00555345520046004726
:109C900000424547494E0052414400442E4D590070
:109CA0005052474D00555345522020200066202039
:109CB0000067202000424547494E202020202000F8
:109CC00052414420202000442E4D592020200043A2
:109CD00020202000081C242C4448586C74050000E7
:109CE00000FFFFFFFF4D000000FFFFFFFF0F000020
:109CF00000F4010000040103010201010411040F3A
:109D0000041704160118010000A59C0000AD9C007A
:109D100000B19C0000B59C00008F9C0000C09C001E
:109D200000C79C0000CF9C0000A09C00000502051D
:109D30000804080B080404050105040908090406C1
:109D400008070206020402060106040701030803CD
:109D5000040C080D020C0203020C010C040D010D91
:109D6000080D040802080807080202070408010891
:109D700004090209010A080B020A0201080A010A81
:109D8000040B01020802041008110210021108104D
:109D90000110041101120212011302130812080F1C
:109DA00008120413011304140214011502150814F7
:109DB0000817081404150115041702170119081AC9
:109DC0000219021602190119041A01160816041BB9
:109DD000021B081A0818021A041B011B0418081891
:109DE000040B042020202020202020202000000020
:109DF0000003000000889C00008D9C00008F9C00E8
:109E000000919C00008F9C0000979C00009B9C0090
:099E100000EB5F0000A09C0000C3
:00000001FF
